:107E9A00424144004032444000403344400040578D
:107EAA004159504F494E5420455849535453400064
:107EBA00205452414E534D4954204552524F52205C
:107ECA0000574159504F494E5400202045584954B3
:107EDA002020210052454345495645004652454512
:107EEA004000454E54455220004D4D2E4D4D4D20DB
:107EFA00004D4D2753532E53005747532138340012
:107F0A002040554054404D402000554054404D00BB
:107F1A00535749535347440050524553454E5440D2
:107F2A00504F532E00414C5400535549405800417C
:107F3A00564700353030003136343000534541520F
:107F4A004348405341545300205D203130404B6335
:107F5A002F70005D2020203140632F2300205D20F8
:107F6A002035404B5453005D203230304046504D4E
:107F7A00004241524F4048454947485400475053F0
:107F8A002048454947485400404947432056414CF8
:107F9A00494400494743405741495420202300415E
:107FAA004C54494043414C202023005550444154ED
:107FBA00494E472E2E0021455849540153454C40FD
:107FCA00524F555445015345542048454947485452
:107FDA0001464C4947485453206869015741595052
:107FEA0054532020686901524F5554455320206844
:107FFA00690153455454494E47536869002145580D
:10800A00495401564152494F20202068690158437A
:10801A002D534554202068690147454E4552414C2D
:10802A0020686901010154455354464C4947485454
:10803A0001534552564345434F4445014641435433
:10804A0052592D5345540021455849540101554E62
:10805A00495401434C49434B40302C4020230143AF
:10806A004F4E5452415354014E4D454121313833FC
:10807A00004C4F43414C00205554432000214558A1
:10808A004954014E455720205741595054014544FF
:10809A0049542057415950540144454C20205741D6
:1080AA005950540101434F4D3A01524543454956EF
:1080BA00452057500153454E4420574159505401C9
:1080CA0053454E4440414C4C40575001014449539A
:1080DA00542057502D57500144454C40414C4C4078
:1080EA005750540021455849540153454C40524F6A
:1080FA00555445014E455720205254455054014588
:10810A0044495420524F55544501524556455253FD
:10811A00452052540144454C2020525445505401A4
:10812A0044454C2020524F5554450101434F4D3A86
:10813A0001524543454956452052540153454E4440
:10814A0020524F5554450021455849540153494E30
:10815A004B212D0153494E4B404D4F440153494E3B
:10816A004B40494E56015445432020204030304070
:10817A0025015641522054434020204023014455B2
:10818A00414C53454E534F520021455849540141E1
:10819A0055544F43454E54014156472F4449535471
:1081AA0001474C44455041544801452D53455420FC
:1081BA0020202E0153544152544C4E450143594CF0
:1081CA00530143594C01545241434B0021455849EC
:1081DA00540152442D45450152442D464C415348C1
:1081EA0001474838300144454C20414C4C20464C0C
:1081FA0000564152494F204E554C4C004B45455074
:0D820A00405155494554403135404D494ED5
:10821700004245464F5245204E554C4C494E47006B
:108227004E4F542150524553454E54004063402011
:108237004B63004654204B6300406340204E4D0083
:108247004654204E4D003022003066004D2F53001B
:1082570057495245004952444100454D5054592011
:1082670052544520004E4F5420454D50545920003C
:1082770053454C21524F55544500214053454C40DE
:108287004C495354002053454C405750544021000B
:10829700204E455740504F534021002140524556EC
:1082A700455253454000214044454C405750545394
:1082B70000214044454C2052544500214053454E2F
:1082C7004440525445002140524543454956454094
:1082D700002020404F204B402020210020204641F5
:1082E700494C202021002045584954003E2145583B
:1082F7004954004C4953540053454E440053544F7E
:1083070052450045444954005940454053004E40AA
:10831700454057005245565253002020555044417E
:1083270054452020004544495420204E45572020DD
:1083370053544F5245004C4F47424F4F4B20454DEA
:10834700505459002145584954015245504C415900
:108357000153454E440144454C4554450021455879
:10836700495401544E432031232035374B01544E95
:108377004320312320392E360101505743403130F5
:10838700234035374B015057434031302340313973
:108397004B01014D5850403130234035374B014D8B
:1083A70058502034232035374B014D585020312366
:1083B7002035374B014D5850403130234031394B30
:1083C700014D58502034232031394B014D5850204E
:1083D70031232031394B005843542D464C494748E7
:1083E7005420003230305E003530305E00312200DC
:1083F700322200332200352200382200464C370053
:10840700464C313600464C333300464C3635004631
:1084170031303000463136300046323630005E2586
:108427002640534F47005E25264054415300414C98
:10843700540056415200225E2F24004B54530041F2
:108447004952434F544543004056322E322D323065
:1084570030354000532F4E004F4646214E4557407A
:108467004D454E55004F46462020202020202020F5
:1084770000475053204552524F520053544F5249D0
:108487004E472E2E0040564152494F400020424150
:10849700524F2000524F55544553004E45415253B9
:1084A700540057415950545300404D41524B53408B
:1084B700004044454C4554454400524F55544500EF
:1084C7004E454152455354004C49535420004252A3
:1084D700472021444953540045544500414C5440DA
:1084E70030002020202141564721202020204453BE
:1084F70054002224004B5400225E004E4D00302CC5
:108507003500312C3000322C3000302C3600312C25
:108517003200322C3500332C3800372C35004031EF
:10852700350040333000403630004C4F4144494E0F
:10853700472E0053455256494345005341543A008C
:108E900012775F128F8F1257EC128F141257F41241
:108EA0008F2102776312775F128F8F1257EC7F5AF0
:108EB000C23C1256CE1258CA783F79437F607EEA90
:108EC000128F831257F47F651256CE1258CA783D1E
:108ED00079417F207E4E128F83303C2012914512C3
:108EE0008FA0783F7943128EFF783D7941128EFF33
:108EF00012914578D7E65480F6753700025C4AC374
:108F0000E796FF1819E796FE0809C3E69FF71819B8
:108F1000E69EF7227F5B7E06907F33124CF51F8022
:108F20000A7F667E147459129F8D1F1255577E3921
:108F3000E4029FAC7866E620E73418C3E694720832
:108F4000E694045029C318E6941F08E69404401ED2
:108F50007869E620E71818C3E6940E08E6940150F5
:108F60000DC318E6947508E694004002D322C3228C
:108F7000E67D0030E7011D08E62BFB18E63CFCE42B
:0E8F80003DFD22C3EB9FF6F71819EC9EF6F7A5
:108F8E0022128F34400CE47842F608F67840F60848
:108F9E00F6227864C3E6946AF55708E6944CF556C3
:108FAE000808C3E69458F55B08E694AEF55A753991
:108FBE0000AC56AD57EC127B0C784C127B9AAC5A27
:108FCE00AD5BEC127B0C7850127B9A7F2B7E867DEC
:108FDE00777C18127AD17850127B8E1279DD127A44
:108FEE00D17850127B8E1279DD127AD17850127BA5
:108FFE008E1279DD127AD17F367E847D257C6412C5
:10900E007AD17850127B8E1279DD127AD1784C1289
:10901E007B8E1279DD127AD17F3F7EA27D607C8BB2
:10902E00127AD17850127B8E1279DD1277CB1277AD
:10903E00CB127BA67F3F7E807D057CE605391279BB
:10904E00DD7848127B9A7F2C7E937D477C7F127A47
:10905E00D17850127B8E1279DD127AD17850127B34
:10906E008E1279DD127AD1784C127B8E1279DD1246
:10907E007AD17F357EB47DF87CDF127AD1785012AA
:10908E007B8E1279DD127AD17850127B8E1279DDB9
:10909E00127AD17F3F7EED7D227CCD127AD1784C33
:1090AE00127B8E1279DD1277CF1277CB7844127B3A
:1090BE009A7F317E397D9D7CE7127AD1784C127B76
:1090CE008E1279DD127AD1784C127B8E1279DD12E6
:0490DE007AD1784487
:1090E200127B8E1277CF127AD17F2C7E377D0C7C49
:1090F200A3127AD1784C127B8E1279DD127AD17852
:109102004C127B8E1279DD127AD1784C127B8E1240
:1091120079DD1277CF127BA67F3F7E807D027C9F16
:1091220005391279DD7844127B9A7848127B8E12C7
:109132007B438E428F437844127B8E127B438E4058
:109142008F4122753900AC42AD43EC127B0C78485A
:10915200127B9AAC40AD41EC127B0C7844127B9AA4
:109162007F2B7E537D507C09127AD17848127B8EF8
:109172001279DD127AD17848127B8E1279DD127A59
:10918200D17844127B8E1279DD127AD17F347EF24D
:109192007DCD7CA3127AD17848127B8E1279DD12B2
:1091A2007AD17848127B8E1279DD127AD17F3F7E96
:1091B2000A7D2E7CAE127AD17844127B8E1279DD32
:1091C2001277CB1277CB784C127B9A7F2B7E4F7D16
:1091D200AF7CB2127AD17848127B8E1279DD127A84
:1091E200D17848127B8E1279DD127AD17848127BBF
:1091F2008E1279DD127AD17F357EB17D4B7C95124C
:109202007AD17848127B8E1279DD127AD1784412A3
:109212007B8E1279DD127AD17F3F7E497DCD7C45EE
:10922200127AD17848127B8E1279DD1277CF1277BB
:10923200CB7850127B9A784C127B8E127B438D55E1
:109242008E568F577850127B8E127B438D598E5AD1
:049252008F5B786452
:10925600E557246AF608E556344CF608E555340415
:10926600F608E55B2458F608E55A34AEF608E43508
:0392760059F62284
:105A960012775F1261291277637F667E00907F140A
:105AA600124CF5125B067F5A78C4125AE2125AEA71
:105AB60078C6125AE2125ACD7F6578C8125AE21297
:105AC6005AEA78CA125AE27E2DE51B129FAC7E3343
:105AD600E51A129FAC7E39E519029FAC860408864A
:105AE60003023C377E15E51C129FAC7E1BE51B129C
:105AF6009FAC7E21E51A129FAC7E27E519029FAC6A
:105B06007F5A7E01E53A129EC27E0B90651DE53BEB
:105B160093029FBFE6FF08E6FE08E6FD339217E410
:105B26005001F4FC127BB775130A753901127DB565
:105B360078D7E6C2E775F00A84F9303D02A9F0127B
:105B46007BB789130539127D8E30170A0539127D08
:105B5600A10539127DA1A803027B9A12775F126113
:105B660029C23C7F5A7E03125A7D125B0612A88711
:105B760010000810011510022080EFE53A146004A9
:105B8600153A8003753A3CD23C80DFE53AB43C05D1
:105B9600753A0180F2053A80EE7E03125A787E0B42
:105BA600125A7D125B0612A8871000081001151004
:105BB600022080EFE53BB40205753B158002153BDC
:105BC600D23C80DFE53BB41505753B0280F2053B10
:105BD60080EE7E0B125A787F5A78C4125AE2125A15
:075BE600EA125C531258DAC9
:105BED0078C4125CAB78C6125AE2125ACD125C859B
:105BFD00751C001258DA78C6125CAB7F6578C81236
:105C0D005AE2125AEA125C531258DA78C8125CAB97
:105C1D0078CA125AE2125ACD125C85751C001258C0
:105C2D00DA78CA125CAB303C14E53B24F4500B78A7
:105C3D00C9E62410F618E63427F6125CB112776324
:105C4D0012545C02A887C2247E15E51C1259CDF5AD
:105C5D001CD2247E1BE51B1259CDF51B1023E77EAC
:105C6D0021E51A1259CDF51A1023E67E27E51912F2
:105C7D0059CDF5191023E822C2247E2DE51B1259AA
:105C8D00CDF51BD2247E33E51A1259CDF51A10230A
:105C9D00E77E39E5191259CDF5191023E622ECF6F8
:105CAD0008EBF62212653578C8E6FE0886073395AF
:105CBD00E0FDFC127AD17FE87E037D007C00127D31
:105CCD00B5127AD178CAE6FE0886073395E0FDFC59
:105CDD00127D8E127AD17F807E697D677CFF127D69
:105CED008EEC127B08127AD17F3F7E807D0D7C1D5C
:105CFD001279DD127AD17F3D7E407D007C00127AD3
:105D0D00D178BC127B8E1279DD127AD17F3E7E80E6
:105D1D007D007C001277CF127AD178BC127B8E1267
:095D2D0079DD127AD17F3F7E80FE
:105D36007D007C001277CB127AD178B4127B8E125A
:105D460079DD127A55783C127B9A7F407E807D0001
:105D56007C00127AD1783C127B8E1279DD127C346B
:105D6600127AD17F3F7EA87D007C00127AD178B866
:105D7600127B8E1279DD1279DD127AD17F407E0098
:105D86007D007C00127AD1783C127B8E1279DD126E
:105D96007C34127AD17F3F7EC07D007C001279DD93
:105DA6001277CF127AD178B8127B8E1279DD127AF9
:105DB600D1783C127B8E1277CF7854127B9A127C64
:105DC6001E7858127B9A127AD11279DD127AD1781E
:105DD600C0127B8E1279DD7844127B9A7854127B3E
:105DE6008E127C34783C127B9A127AD11279DD12AB
:105DF6007AD178BC127B8E1279DD783C127B9A7F41
:105E06003E7EC07D007C00127AD1783C127B8E12D9
:105E160079DD127AD17F3F7E007D007C001277CF3C
:105E2600127AD1783C127B8E1279DD127AD17F3FBD
:105E36007E807D007C001277CF127AD178B4127BF7
:105E46008E1279DD7870127B9A78C4E6FE08860792
:105E56003395E0FDFC127AD17FE87E037D007C005D
:105E6600127DB5127AD178C6E6FE0886073395E02C
:105E7600FDFC127D8E127AD17FE07E5E7DF87CFF7E
:105E8600127D8EEC127B08127AD17F3F7E7F7DE5F4
:055E96007CC9127AD165
:105E9B007870127B8E1279DD127A557850127B9ABC
:105EAB007F3F7EF07D007C00127AD1783C127B8E96
:105EBB001279DD127AD17F3F7EC07D007C00127794
:105ECB00CF127AD1783C127B8E1279DD127AD17F88
:105EDB003F7E807D007C001277CF783C127B9A78D6
:105EEB00BC127B8E127AD17F3F7E807D007C0012AC
:105EFB0077CB127AD1783C127B8E127AD178B4128E
:105F0B007B8E1279DD1279DD7840127B9A785412F0
:105F1B007B8E127C6C783C127B9A127AD11279DDD3
:105F2B007874127B9A7F417E107D007C00127AD1AF
:105F3B0078C0127B8E1279DD127AD17F407E807D04
:105F4B00007C00127AD17844127B8E1279DD127AA2
:105F5B00D17F417E207D007C001277CB127AD178E5
:105F6B0044127B8E1279DD127AD17F407E407D0008
:105F7B007C00127AD17874127B8E1279DD127AD171
:105F8B007F407EA07D007C001277CF1277CF1277F7
:105F9B00CB127AD17850127B8E1279DD127AD178AE
:105FAB0050127B8E1279DD127AD17F3D7E2A7DAA2B
:105FBB007CAB1279DD127AD17F3F7E007D007C00B5
:105FCB001277CB127AD1783C127B8E127AD1787001
:105FDB00127B8E1279DD127AD17840127B8E127A77
:105FEB0055127AD17850127B8E1279DD127AD178D4
:105FFB0050127B8E1279DD1279DD127AD178541220
:0C600B007B8E1277CB127AD17F4A7E5137
:106017007DD27CCB1279DD127B4378AC127B9A7FE1
:10602700407E007D007C00127AD17874127B8E123C
:1060370079DD127AD17F3F7E807D007C001277CF99
:10604700127AD17844127B8E1277CF127AD1785098
:10605700127B8E1279DD127AD17850127B8E1279EB
:10606700DD127AD17850127B8E1279DD127AD17FC8
:106077003E7E2A7DAA7CAB1279DD127AD178501246
:106087007B8E1277CB127AD17858127B8E127A5583
:10609700127AD17F4A7E517DD27CCB1279DD127B79
:1060A70043127AD1AF3AEF3395E0FEFDFC127AD175
:1060B7007F407E7E7D057C00127DB5127AD17F60A0
:1060C7007E757D587CFF127D8E127D8E78B0127B97
:1060D7009A78AC751B641261008F1C78B0751B67CA
:1060E700126100E51C75F00AA42FFF249C50027F63
:1060F7000078D7E654802FF622753900127B8E126E
:106107007AD17F0A7E007D007C00127E61A81BE5A4
:1061170013F608E512F608E511F6335004EFF40418
:10612700FF22C23D78647BAC125B1AD23D78677B55
:10613700B0125B1A1265357F007EE47D577C001232
:106147007AD178AC127B8E127D8E127AD17F007E47
:0E615700537D077C00127E61127AF085133BA7
:106165007F807ECB7DA47C00127AD178B0127B8EA5
:10617500127D8E127AD17F407E7E7D057C00127E57
:1061850061127AF0E513F56F04F53A85126E851103
:106195006D85106C7F407E7E7D057C00127AD178FE
:1061A5006C127B8E127DB5127AD17F607E0C7DA23A
:1061B5007C00127AD178B0127B8E127D8E127DA171
:1061C500786C127B9A78AC127B8EEC127B08127A73
:1061D500D17F347E9C7D2B7C5F1279DD7854127BD8
:1061E5009A127C1E7850127B9A786C127B8EEC1278
:1061F5007B08127AD17F347E9C7D2B7C5F1279DD02
:10620500127AD17850127B8E1279DD7840127B9A02
:106215007F407E007D007C00127AD17854127B8EFF
:106225001279DD127C34127AD17F3D7EC07D007CEF
:1062350000127AD178BC127B8E1279DD127AD17F69
:106245003E7EC07D007C001277CF127AD178BC12D9
:106255007B8E1279DD1279DD127AD17F3D7E407D0C
:10626500007C00127AD178BC127B8E1279DD127A0D
:10627500D17F3E7E807D007C001277CF127AD17867
:10628500BC127B8E1279DD127AD17F3F7E807D0034
:106295007C001277CB127AD17854127B8E1279DD7D
:1062A5001277CB127AD17F407E807D007C00127AF6
:1062B500D17854127B8E1279DD127C34127AD17F1B
:0F62C5003D7E707D007C00127AD178BC127B8EFA
:1062D4001279DD127AD178BC127B8E1279DD1279B3
:1062E400DD1277CF127AD178B4127B8E1279DD78F1
:1062F40058127B9A7854127B8E127C34783C127B31
:106304009A7854127B8E127C6C7854127B9A783C67
:10631400127B8E127AD11279DD127AD178BC127B7B
:106324008E1279DD783C127B9A7F3E7EC07D007CA4
:1063340000127AD1783C127B8E1279DD127AD17FE9
:106344003F7E007D007C001277CF127AD1783C1218
:106354007B8E1279DD127AD17F3F7E807D007C00B6
:106364001277CF127AD178B4127B8E1279DD7870DD
:10637400127B9A7850127B8E127AD11279DD127ABE
:10638400D178C0127B8E1279DD7844127B9A7854CE
:10639400127B8E127AD11279DD7874127B9A78404E
:1063A400127B8E127AD11279DD783C127B9A7F406F
:1063B4007E807D007C00127AD17844127B8E127923
:1063C400DD127AD17F417E107D007C001277CF12DE
:1063D4007AD17844127B8E1279DD127AD1787412D4
:1063E4007B8E127AD17F407EA07D007C001277CB19
:1063F4001277CF127AD1783C127B8E1279DD127A21
:10640400D17F3D7E2A7DAA7CAB1279DD127AD17FC1
:106414003F7E007D007C001277CF127AD17854122F
:106424007B8E127AD17870127B8E1279DD127AD13A
:10643400783C127B8E1279DD1279DD127AD178588C
:10644400127B8E1277CF127AD17F3F7E7F7DE57CDF
:01645400C97E
:106455001279DD127AD17F4B7E187D967C8012777A
:10646500CF127B43127AD17FE87E037D007C001238
:106475007E61127AF078C8A61208A61308A6060847
:10648500A6077874127B8E127AD17F3F7E807D00BD
:106495007C001277CB127AD17844127B8E1277CF9B
:1064A500127AD17F3E7E2A7DAA7CAB1279DD127AE3
:1064B500D17840127B8E1279DD127AD1783C127B2D
:1064C5008E1279DD127AD17840127B8E1277CF1237
:1064D5007AD17F3F7E7F7DE57CC9127AD1787012B3
:1064E5007B8E1279DD1279DD127AD17F487EF47DBB
:1064F500247C001277CF127B43127AD17FE87E038A
:106505007D007C00127E61127AF078C4A61208A67E
:106515001308A60608A607223F3F434445464748B9
:106525004A4B4C4D4E5051525354555657583F3F78
:10653500E4F539F5A7906549791078B4E493F6A3A5
:1065450008D9F92232A5C24A4A19DC3A885CDB3BF4
:04655500FFD6DC3B56
:10775F00D2D58002C2D575A70490040078107F0B94
:10776F0012778B78267F0512778B783C7F221277E2
:10777F008B786A7F0F12778B75A7002230D506E6BC
:10778F00F008DFFB22E0F608DFFB22D2D58002C231
:10779F00D575A7049006FA78737F0612778B75A7B5
:1077AF000022DA0CD902800BD906303701B350050D
:1077BF0002793E923702792AD9F680F9D2368002C1
:1077CF00C23612796F303606C86002B237C89236A9
:1077DF00DAD0D9E4B8000A1279B6A2369237027914
:1077EF001360FBB51300400F1279B6A23692F7A2C1
:1077FF00379236A2F79237C398F40424E740DF2478
:10780F0019AD29AC28AB277A00C394084008CDCC1A
:10781F00CBCAE4CD80F424086010F9C3ED13FDEC5E
:10782F0013FCEB13FBEA13FAD9F1A236303701B38D
:10783F0040308A17E5102BF518E5113CF519E512C4
:10784F003DF51A501A13F51AE51913F519E5181322
:10785F00F518E51713F5170513E513700205140254
:03786F0078C9E4F1
:10787200C39AF517E5109BF518E5119CF519E51269
:107882009DF51A500DB237C378177F04E496F608B7
:10789200DFFA7A047019E513C39408F51350021540
:1078A20014E4C517C518C519F51ADAE802796A2071
:1078B200E7BAE5137002151415137817C37F04E6AF
:1078C20033F608DFFA80E8E51A20E7137817C37F5A
:1078D20004E633F608DFFAE513700215141513E512
:1078E200173378187F03E63400F6500E08DFF77579
:1078F2001A800513E51370020514E51420E754708D
:1079020027E513604E046020851A12851911851827
:10791200105326F0AC10AD11A237E51313FFE51298
:1079220092E7FEA813027AF0E4F512F511F510F5CC
:10793200147513FF5326F043260580D8E5FFF51290
:10794200F511F510751400F513D2375326F04326BE
:107952000980C15326F0432603E4F512F511F51010
:10796200F514F513C23780AC5326F080EC79017A16
:10797200018512F0E513A2F7339237751400F5135F
:107982006002D2F785F012A813B8FF0809E512C207
:01799200E70D
:107993006001098C278D288EF0A2F7EF3304700A5B
:1079A3000AC2F705F00AD5F0011A146002D2F7856E
:1079B300F02922C88813C512C529C512C511C528C7
:1079C300C511C510C527C51022DA03B80003027913
:1079D3003ED9028002D9F702792A12796F30370132
:1079E300B392377004D9E78005DADEB80003027971
:1079F3006AD9E2C3947E500215142513F51350027D
:107A030005147815760008B81BFA78277915E60867
:107A1300FAE8FC78108AF0E608A427F709E5F037BE
:107A2300F7500989F00907E760FBA9F0B813E619D5
:107A330019ECF8B82AD80278C9027955B8FFFA02C6
:107A4300793ED9FB02792ADAF6B800F002796A1294
:107A53007BA612796F303701B392377007D9E3B839
:107A630000E280DBDAE1B8000280E1D9D5C8C3982F
:107A730050021514247F50020514F513781A76006A
:107A83007A1A7B80C3E5109527E5119528E51295B1
:107A9300294016C3E5109527F510E5119528F51132
:097AA300E5129529F512E64BF6F7
:107AAC00DA030278C9EB03FB30E703187600C3E571
:107ABC001033F510E51133F511E51233F51240CA08
:107ACC0030E7DD80B6E53905396010D0F0D0E0C084
:107ADC0010C011C012C013C0E0C0F08F138E128DF5
:107AEC00118C1022E539146010D0F0D0E0D013D0F6
:107AFC0012D011D010C0E0C0F01539227920800CC2
:107B0C007910800479087D007E007F003392D55077
:107B1C0003127B80EC33400FEF33FFEE33FEED337B
:107B2C00FDEC33FCD9EE22EECCF5F0747E29A2D517
:107B3C0013FF92F7AEF022EF8EF0A2F7D2F733924A
:107B4C00D5C3947F5006E4FFFEFDFC229420400434
:107B5C0074FF80F304CCFEE4FFFAE5F0CC6012C3B2
:107B6C00CC13CCCD13CDCE13CECF13CF0450EEDA35
:107B7C00EC30D5D7C3E49FFFE49EFEE49DFDE49C6E
:037B8C00FC22E6F2
:107B8F00FC08E6FD08E6FE08E6FF22ECF608EDF637
:107B9F0008EEF608EFF622CFC513CFCEC512CECD25
:107BAF00C511CDCCC510CC22E4F513F512F511F5A6
:107BBF001022E493FCA3E493FDA3E493FEA3E493C8
:107BCF00FFA322C0E0127AD11279DD127C05127B5D
:107BDF00C1D0E0C0E0127AD1127BFC1279DD127AAB
:107BEF00D1127BC11277CFD0E0D5E0E722AC48AD00
:107BFF0049AE4AAF4B228C488D498E4A8F4B227427
:107C0F00FF7809FFFEFDFCE52654F048F526221209
:107C1F007CC504A2E1927F1420E015907D46740488
:107C2F00127BD28029127CC530E102B27F20E0EBBB
:107C3F008C4C8D4D8E4E8F4F907D5A7404127BD28B
:107C4F00127AD1AC4CAD4DAE4EAF4F1279DD307FC5
:107C5F0004EF6480FFEE33EF337001FF22127CC517
:107C6F00C0E08C4C8D4D8E4E8F4F907D7E740312E5
:107C7F007BD2127AD1AC4CAD4DAE4EAF4F1279DDF7
:017C8F00EC08
:107C9000C54CFCEDC54DFDEEC54EFEEFC54FFF904A
:107CA0007D6E7403127BD2D082127AD1AC4CAD4D72
:107CB000AE4EAF4FE58230E007127A55B27F809D1D
:107CC000127A528098EE33EF3324605007D0E0D020
:107CD000E0027C0EEFA2E7547F927FFF127AD17C04
:107CE000837DF97E227F3E1279DDEE33EF332481EE
:107CF0005010127AD1127B43127B08EFB2E7FF12C9
:107D000077CFEE33EF33602A2403F8C313FFEE92EC
:107D1000E7FEE82481E4501A127AD1127B43EF0483
:107D2000C2E0FCF582127B10EFB2E7FF1277CFE5DD
:107D30008203FAEE33EF33600B148FF0A2F713FFD8
:107D4000EE92E7FEEA2283FA703AE4E9AABCF8E090
:107D5000813EE6E99DBF0000803F1A3C28396669F4
:107D600099BBE335A33DE75D25BFDB0FC93FCCDB06
:107D70008D41EE3649C43F91C9453DF8B0C500007C
:107D8000803F34F517C373FA2F45DDFD0AC6EF2592
:107D900013FFEE3512FEED3511FDEC3510FC027AC5
:107DA000F0C3EF9513FFEE9512FEED9511FDEC95E6
:107DB00010FC027AF0EFF88513F0A4FFE513C5F08C
:0A7DC000CEF9A42EFEE435F0CDFA52
:107DCA0088F0E512A42EFEED35F0FDE433CC8513E0
:107DDA00F0A42CFCE5128AF0A42CFCE51189F0A48D
:107DEA002CFCE51088F0A42CFC89F0E512A42DFDEA
:107DFA00EC35F0FCE51188F0A42DFDEC35F0FC8A99
:107E0A00F0E513A42DFDEC35F0FC027AF0E4CCF891
:107E1A00E4CDF9E4CEFAE4CFFB75F020C3E51333E1
:107E2A00F513E51233F512E51133F511E51033F5C3
:107E3A0010EF33FFEE33FEED33FDEC33FCEF9BEE38
:107E4A009AED99EC98400CFCEF9BFFEE9AFEED99A7
:107E5A00FD0513D5F0C622C2D5EC30E705B2D5121E
:107E6A007B80E51030E70DB2D5127E84127E1712A0
:107E7A007B808003127E1730D515C3E49513F51362
:107E8A00E49512F512E49511F511E49510F5102216
:106F9700E57124885002D219123FC0126F7712454B
:106FA700261244C41267F3124429122A131233A873
:106FB700103626301219E41270CB1270E01271DF0E
:106FC70012720130510302728B12755C205109C293
:106FD70051E4F552F545F5442274FF1270CB7873EE
:106FE7007973123FD48F1C8E1B7510DF751100E566
:106FF7001164B470061270967511101270634028F0
:10700700AF1CAE1B12422720321EAC03AB027A0C18
:10701700123C6FED701275A700758304851182EC21
:10702700F00583E510F00511D510C412709675C7E9
:107037000375C6E075A7049005007F04127051DF41
:10704700FB75A700121D6F0244C4E0F5BCE0F5BD57
:10705700E0F5BEE0F5BF1239E405C622E51075F08C
:1070670004A4F5C685F0C775B901E5BC33401F0513
:10707700C605C675B90185BE6485BF6505C675B900
:107087000185BC6685BD6785BE6885BF69C322E586
:107097001124FE502E75A7007F10AE111E758304B4
:1070A7008E82E0FD1582E0CDB505005012F0058215
:1070B700CDF00583E0FD1582E0CDF00582CDF0DE51
:1070C700DCDFD72275A75490040005A79005007F41
:0370D700B4F0F022
:1070DA00DFFC75A70022128CA2C2517B077AFFE45B
:1070EA00FFF5A79004001271C3ED244C403275A736
:1070FA00008D8205A71271897583058D82E024109F
:10710A00401CF005A7E02CF0500505A7E004F0BAF2
:10711A00000CBB0009D251EF24DC50027F23DFC6EA
:10712A00EA600512713C8006EB600312717475A760
:10713A00002230E0047553082230E1047553182206
:10714A0030E2047553282230E3047553382230E4C0
:10715A00047553482230E5047553582230E6047505
:10716A0053682230E7037553782230E00475538858
:10717A002230E1047553982230E2037553AA22EDB6
:10718A0054F0C42323907193735302FE225302FDD9
:10719A00225302FB225302F7225302EF225302DF49
:1071AA00225302BF2253027F225303FE225303FDBE
:1071BA00225303FB225303FB22128BCD128ACAE409
:1071CA00F5F7C2B2C2B2ADF7F5F7C2B2C2B2ACF7C6
:1071DA00D2B2C2202290050078B4E06015FD54F0C6
:1071EA00C4CD7C00540FFE1583E0FF123D6DEFF015
:0771FA0005830582D8E422A1
:1072010075830478FF088882E060FAF5D38812E577
:1072110012244C50012285D3D288D4881279FF05DB
:1072210012E51260F00908E875F0B484A8F08882CC
:10723100E060ECF5D3B9000280D5B9230050D0C38A
:1072410095D292D15002F40409FEE4FFFCAD011283
:107251003D7A7401FA25D475F0B484A8F0AC06AB7C
:1072610007123C61EB30E7010CE5D22C30D1029CD6
:107271009C8882F00AEAB501DCE512244C50012217
:1072810085D3D28512D4A812809390040012734A38
:107291008C068B0512734AE4FFF512F5118C148BE1
:1072A10013C3ED9BF9EE9CFA4012E51199E5129A90
:1072B100500A8C148B138A1289118F528F82E0F934
:1072C100C3ED99FDEE9400FEE582245A5002244C50
:1072D10075F0B48485F082E0FA2DFDEE3400FEEB0A
:1072E1009AFBEC9400FCE92BFBEC3400FC0FBFB4DF
:0E72F100B0E55224D3400224B4F552C3E51395
:1072FF0033FBE51433FCE511FE2BFBE512FF3CFCE1
:10730F00123DCFE9F890735C93F511FDEBF513FF88
:10731F00ECF514FE7C00123D6D8F44E890745C9385
:10732F00FAAB13AC14123C98AF03AE04AD117C0052
:10733F00123D6DEF7002F552F545227C007B007F08
:10734F005AE02BFBEC3400FC0582DFF522B4B4B419
:10735F00B4B4B4B4B4B4B4B4B4B4B4B4B4B4B4B3DF
:10736F00B3B3B3B3B3B3B3B3B3B3B3B3B2B2B2B2E2
:10737F00B2B2B2B2B2B1B1B1B1B1B1B1B0B0B0B0ED
:10738F00B0B0B0AFAFAFAFAFAEAEAEAEAEAEADAD05
:10739F00ADADADACACACACACABABABABAAAAAAAA27
:1073AF00A9A9A9A9A9A8A8A8A8A7A7A7A7A6A6A653
:1073BF00A5A5A5A5A4A4A4A4A3A3A3A2A2A2A2A188
:1073CF00A1A1A0A0A0A09F9F9F9E9E9E9D9D9D9DC1
:1073DF009C9C9C9B9B9B9A9A9A99999999989898FF
:1073EF009797979696969595959494949393939241
:1073FF009292919191919090908F8F8F8E8E8E8D82
:10740F008D8D8C8C8C8B8B8B8A8A8A8989898888C5
:10741F00888787878686868585858484848383830A
:10742F008282828181818080807F7F7F7E7E7E7E4F
:10743F007D7D7D7C7C7C7B7B7B7A7A7A7979797890
:10744F00787877777776767675757574740002032A
:10745F00050608090B0C0E101113141617191A1C18
:10746F001D1F2122242527282A2B2D2E303133347E
:10747F003637393A3C3D3F404243454648494B4CED
:10748F004E4F505253555658595A5C5D5F60616369
:10749F00646667686A6B6C6E6F70727374767778F8
:1074AF007A7B7C7E7F80818384858688898A8B8D99
:1074BF008E8F9091929495969798999B9C9D9E9F55
:1074CF00A0A1A2A4A5A6A7A8A9AAABACADAEAFB028
:1074DF00B1B2B3B4B5B6B7B8B9BABBBCBDBEBFC015
:1074EF00C0C1C2C3C4C5C6C7C7C8C9CACBCCCCCD1F
:1074FF00CECFD0D0D1D2D3D4D4D5D6D7D7D8D9DA3E
:10750F00DADBDCDCDDDEDEDFE0E0E1E2E2E3E4E477
:10751F00E5E5E6E7E7E8E8E9EAEAEBEBECECEDEEC8
:10752F00EEEFEFF0F0F1F1F2F2F3F3F4F4F4F5F52E
:10753F00F6F6F7F7F8F8F8F9F9FAFAFAFBFBFBFCAD
:10754F00FCFDFDFDFEFEFEFEFFFFFFFFFFC251E44F
:10755F00F544F814FB900400A9007C0FC2D11276F9
:10756F0077E82405F8B8B4F08B13E5122403FA2456
:10757F004C5001FABBFF012275112C8A191276AEFD
:10758F008F16203D12AA197511231276AE8F15751D
:10759F001600303DE28011751123127656751500D5
:1075AF00303D05E82F13F515751112127656751427
:1075BF0000303D05E82F13F514EA2404F552244C4E
:1075CF005002F552E4F51AF51BF51CE516600AFB9F
:1075DF007A00AF137EFF12761CE515600AFB7A4F17
:1075EF00AF137EFF12761CE516600DFB7A00E514D3
:1075FF006006FF7ECF12761CAE1CAF1B7C00AD1A4F
:06760F00123D6D8F45EFF6
:107615002513F544D25122EFF5F0A4FCADF0EBF5BE
:10762500F0A49CFCE5F09DFDEB8AF0A4FAABF0EF2D
:107635008EF0A49AF8E5F09BF9E833F8E933F97B85
:1076450000123E13051AE51B2BF51BE4351CF51C32
:1076550022EA2511F9244C5001F9C2D11276753070
:107665003D428F00C3EA9511F9500324B4F9D2D1F4
:107675007C09E4FDFEFF8982E060062FFFE43EFE03
:107685000D09B9B4027900DCEDED20D118F51E2401
:10769500FE923D500F123D7AEFB503005006851E50
:1076A5001FFB881222F51D80E6127656203D437495
:1076B5000212774D127656203D3874041277551212
:1076C5007656203D2D740612774D127656203D22B2
:1076D5007408127755127656203D17740A12774DA5
:1076E500127656203D0C740C127755127656203DB5
:1076F5000122C3E89F605088148F158A1640081A26
:10770500BAFF0A7AB380060ABAB4027A001276562C
:0E771500303D34C3E89FF9602EC3E51495158E
:10772300FB6930E7D4E930E703F404F9EB30E7020F
:10773300F404C3995002AA16E5142515C82F28FF8F
:10774300E4FC33FE7D04123D6D222AFA244C5001E1
:0C775300FA22C3CA9AFA500324B4FA22A6
:108A3B00C2B212A9BDD2B275F83022C2B2F5F7C2DA
:108A4B00B2C2B2D2B222D220D2147406128A4674A7
:108A5B00C7128A46120656128A6E1239E4801F74A8
:108A6B00FF8001E4F5BCF5BDF5BEF5BF221206563D
:108A7B0085BF6C85BE6B756A00128AE7C21FD22058
:108A8B00C2B275F705C2B2C2B2C2B2C2B275F705B5
:108A9B00C2B2C2B2C2B2C2B2E5F7540170EFD2B2E7
:108AAB00C22022D220C2B2F5F7C2B2C2B2856CF795
:108ABB00C2B2C2B2856BF7C2B2C2B2856AF722D21A
:108ACB0020C2B275F703C2B2C2B2856FF7C2B2C28F
:108ADB00B2856EF7C2B2C2B2856DF722E56B701725
:108AEB00E56A7013D220128A897406128A4674D8EA
:108AFB00128AAED2B2D21FC22022128A89D220741D
:108B0B0006128A467402128AAE8FF7C2B2C2B2D272
:108B1B00B2C22022852E72E55F030354C0F8E55ED6
:108B2B00543F28F57C30550122201F06128AE7306E
:108B3B001F25D220C2B275F705C2B2C2B2C2B2C2F1
:108B4B00B275F705C2B2C2B2C2B2C2B2E5F75401F6
:108B5B00D2B2C220600122C21F128DCE128A89D2DC
:108B6B00207406128A467402128AAE787086F70851
:108B7B00B880FAD2B2C2207410256A54F0F56AE4B8
:108B8B00356BF56BE4356C540FF56C22E56A2401FB
:108B9B0080EBD380EAE54B75F010A4256A54F0F511
:108BAB006AE5F080DBE56A24F054F0F56AE56B3496
:108BBB00FFF56BE56C34FF80CEE56A24FF80ECC3D8
:108BCB0080EBE56D24F054F0F56DE56E34FFF56E3A
:108BDB00E56F34FF540FF56F22D3E4356EF56EE479
:108BEB00356F80F0128C49128C75C254C255E57FDB
:108BFB007002D255147002D254E54A30E00122B40F
:108C0B00061E20540F128BB0128D19128DAD128DC2
:108C1B00E5028E6112655F7E0412A9B9754A0122C5
:108C2B0020550F128B82128D8C128DCE128CF2026C
:108C3B008E3412655F7E0412A9B9754A052274033E
:108C4B00128AAE7870E4F5F7C2B2C2B2A6F708B8D2
:108C5B0080F3D2B2C220227403128AAEE4F5F7C2BB
:108C6B00B2C2B2E5F7D2B2C22022E575F8541F307A
:108C7B00E40244E0F57585722EA2779226E57C54CA
:108C8B003F30E50244C0F55EE57C54C02323F55F1D
:108C9B00E57F1414F55122856C6F856B6E856A6DBB
:048CAB0022856F6C43
:108CAF00856E6B856D6A22E4FEFF740775A704F568
:108CBF00838E8274FFF0DFFD75A7002274067E009D
:108CCF007FB0128CBBE4F55AF55B2275A704758350
:108CDF0006E55A600A75F00A84E5F07002740AC45A
:108CEF00F58222307720E55A24024002055A128C71
:108CFF00DAE55AF0E573F0E574F0E575F0E576F036
:108D0F00E577F0E578F075A700223077F9128CDA65
:108D1F007F1074FFF0DFFDE55A24F55003128D44E8
:108D2F00155AE55AB4FF02055AC3E55A955B50D65A
:108D3F00755B0080D1128CA27F0A056D056D128ABA
:108D4F00CAE4F5F7C2B2C2B2E5F7D2B2C22030E739
:108D5F0004DF028005128BCD80E0056D128ACA12E6
:108D6F008CDAE55A24F6F07F06E4F5F7C2B2C2B208
:108D7F00E5F7F0DFF4D2B2C22075A70022053FE578
:108D8F003FB43C17753F00053EE53EB43C0D753EC4
:108D9F0000053DE53DB41803753D0002362B153F28
:108DAF00E53FB4FF17753F3B153EE53EB4FF0D752C
:108DBF003E3B153DE53DB4FF03753D1702362B05D0
:108DCF0042E542B43C0F7542000541E541B43C0514
:0A8DDF007541000540221542E542EF
:108DE900B4FF0F75423B1541E541B4FF0575413BA1
:108DF900154022E54075F03CA42541FBE435F0FC23
:108E09007A3C123C61EB2542FBE43CFC22E53D75D2
:108E1900F03CA4253EFBE435F0FC7A3C123C61EBC6
:108E2900253FFBE43CFC2220740122C3E5709557E1
:108E3900FF24FD5021EF24EB400A78BD06B6001649
:108E490018068012EF2402400DEF2414500878BB55
:108E590006B600021806802BC3E5709557FF24FD5E
:108E69005021EF24EB400A78BB16B6FF161816807E
:108E790012EF2402400DEF2414500878BD16B6FFF6
:078E89000218168570572244
:10A9AC0012A9AF7E0480067E0280027E017F0080A9
:10A9BC00047F017E00EF4E6012E4FD0D1D0DEDC312
:0CA9CC0094AD40F7EF1F70ED1E80EA22F2
:10AA4400D22FF5D8D2DCE5F520E7FBE5DA540FFE8A
:06AA5400AFD975D8002205
:10A6A4007F767E0690A70D124CC4740412AA447CD3
:10A6B400007D52123D6DEFF875F00A84C0F07F768C
:10A6C4007E23129FAC7E29742E129FBF7E2ED0E073
:10A6D400129FAC7E357456129FBF7F6B7E1190A77C
:10A6E40012129FEDE824E04001220423F824E750ED
:10A6F40002781812A6FDD8FB227F6CE82411FE799B
:10A704000512A94C0E0FD9F9224143435500071DE8
:10A71400FFFFFFE080000020C0000038E0000008D8
:0CA72400F0000038F8000020FFFFFFE00C
:10A7B20012A7DA30E6022409540F75F00AA4F5153F
:10A7C20012A7DA30E6022409540F25152212A7DA5D
:10A7D200540F2275F0BE800D75F022800875F007C7
:10A7E200800375F004E4206D07D5E0FAD5F0F72276
:10A7F200C2ACE54F623885504F8599509247A26EA0
:10A80200926DA26F926EC26FA247D2AC2212A819A9
:10A81200C4FA12A8192A2212A7DA20E603540F2238
:05A82200540724092287
:10A73000E612A73718E608FAC412A73DEA540F44F8
:10A7400030F924C6E9501624078012753800800DB0
:10A7500075F00A84C0F012A75BD0E0443030530992
:10A7600075F00085E0E0D5F0FA3099FDC299F599D1
:10A77000623822E53880F2753800744012A75D74A3
:10A780002A12A75D6238633840E53812A73780087F
:10A7900012A75DE53812A75D740D12A75D740A80DB
:10A7A000BC744012A75D744080B3742C80AF742ECB
:02A7B00080AB7C
:10AA6C0085A0835383FE438380858384F0758400A3
:01AA7C0022B7
:10A4E70074A212AA6C74A112AA6C74C012AA6C741A
:10A4F7002512AA6C12A56975C70375C6FC75B90143
:10A5070012A53A24EA50027E16EE90A5529325BC76
:10A51700FE24E6501A24E84016748112AA6CEE1243
:10A52700AA6C12A576742F12AA6C74AF02AA6C7E5D
:10A537002680E6740812AA44EE75F020A4FEEF54B4
:10A54700F80303032E2492C313FE22F7F7F8F8F952
:10A55700FAFBFCFDFEFF00000000010102020203FE
:10A567000303A8BCA9BDAABEABBFACC7ADC62288B2
:0CA57700BC89BD8ABE8BBF8CC78DC6227C
:10A88700D21AC006C007C0E075A7019000007EB7C6
:10A8970075A700EE12AA6C741012AA6C740412AA9F
:10A8A7006C85A08343838185838475A7517F80E06E
:10A8B700F0DFFC1EBEAFD9E4F5A7F584D0E0D007E2
:05A8C700D006C21A22B8
:10AA5A0075A711900000E4C583F0C58330E2F8F5CC
:02AA6A00A72221
:10A94C00EF20E723EE20E71F20E61C05A7C45403E5
:10A95C00F583EE5408C42FF582EE5407240983F5D1
:10A96C00F0E045F0F005A722804020100804020119
:10A97C00EF20E723EE20E71F20E61C05A7C45403B5
:10A98C00F583EE5408C42FF582EE5407240983F5A1
:10A99C00F0E055F0F005A7227FBFDFEFF7FBFDFEDF
:109F6C00FDA42582F582E5F03583F583ED22904939
:109F7C00237A0475F005129F6C7D0580607A05804C
:109F8C00027A04547FC0E0C083C082C39420500185
:109F9C00E49048D3129F7F8030904A2C7A0580053C
:109FAC00904AE27A0675F007129F6C7D07802E7A34
:109FBC000580027A06547FC0E0C083C082C394201F
:109FCC005001E4904A72129FB1D082D083D0E0222B
:109FDC0090485175F00A129F6C7D0A7A07C2D180A5
:109FEC0002D2D1C0A7C082C083C007C006C0E03077
:109FFC00D10975A704E493FDE493FAEEFB75A7046D
:10A00C00EBFEEAFC7901D9067908E493F5D4E5D4A2
:10A01C0023F5D420E01612A97C0EDCEA0FDDE1D08A
:10A02C00E0D006D007D083D082D0A72212A94C80D2
:10A03C00E890479175F00E129F6C7D0E7A08129F76
:10A04C00E990483975F002129F6CE493FDE4A393F8
:10A05C00FACE2408CE7C0812A06A7C06AD02ED2351
:10A06C00FD20E00712A97C0FDCF42212A94C80F72A
:109E5700F5D2C2D58036F5D2D2D58030F5D224F6E8
:109E670050090E0E24A650030E0E0EE5D2F5D2753C
:109E7700F0648485F0D3C2D57009D2D57420129FBF
:109E8700BF8003129FACCE2406CEE5D375F00A84BB
:109E970085F0D3700A30D5077420129FBF80031254
:109EA7009FACCE2406CEE5D3129FACE5D222F5D2E5
:109EB70075F0648485F0D3C2D58022F5D2C2D580EF
:109EC70025F5D2D2D5801FF5D275F0648485F0D3FD
:109ED700C2D57009D2D57420129FBF8003129FA5E7
:109EE700CE2405CEE5D375F00A8485F0D3700A3009
:109EF700D5077420129FBF8003129FA5CE2405CEDD
:109F0700E5D3129FA5E5D222F5D2C2D58035F5D289
:109F1700D2D5802F30E70DF404C0E0742D129F8D49
:109F27000E0ED0E0F5D275F0648485F0D3C2D570FB
:109F370009D2D57420129F8D8003129F7ACE2404F4
:109F4700CEE5D375F00A8485F0D3700A30D507744F
:109F570020129F8D8003129F7ACE2404CEE5D31260
:059F67009F7AE5D22203
:104CB000D23C8002C23C7405FEF51EE4FFF51DF5F2
:104CC0001F203C3175A700E493700122A3B40204B5
:104CD000051D8003B4010A051FEF2409FFAE1E80E5
:104CE000E6129FBF7D06B440027D03B421027D021F
:104CF000EE2DFE80D275A700E493700122A3B402CA
:104D000004051D8003B4010F051FEF2407FFAE1E2D
:104D100080E6129F898008B45B0050F6129F8D0ECA
:104D2000B4210280D30EB4400280CDB42C0280C8DE
:104D30000E0EB45F0280C1B45B0040BC0E0E80B8A2
:104D4000E608129FBFEE2406FED513F422E60812F1
:104D50009F8DEE2404FED519F422907E9A307409BA
:104D6000907E9E307303907EA3024CC475F019D5DB
:104D7000E0FDD5F0FA1233EE12A7A1744F12A74B43
:104D8000744B02A790124DC31233EED2AC12A7D5CA
:104D9000C5F06024C5F0B440F412A7DAB4400312A1
:104DA000A7DAB44F1A12A7DAB44B1412A7DA12A773
:104DB000DA12A7DAC2ACC32212A7D5C5F070D5C2E9
:104DC000ACD32230530975F008D5E0FDD5F0FA22B6
:104DD0007F0375F019D5E0FDD5F0FA1233EE12A776
:104DE000A1745712A74B745012A75D748112A75D6E
:104DF000E56312A75DE56212A75D78D0E612A75DB4
:104E000008B8D7F8E6F8795F30E702792FE912A7FA
:104E10005D12A75D12A75D12A75D745812A75D749D
:104E20004312A75DE412A75DE8C2E775F00A84C4E7
:104E300025F012A75D7864E612A75D08B869F8E668
:104E400012A790124D85400122DF02800775F00005
:104E50008083D250C2ACD322124DC3C2501233EE63
:104E6000D2AC2002EF12A7D5C5F060E6C5F0B44081
:104E7000F112A7DAB4400312A7DAB457D7F5381203
:104E8000A7DAB450CF12A7DA12A7DAF56312A7DABD
:104E9000F56278D012A7DAF924A0500353015FE934
:104EA00024E04002795FA60108B8D8E8780612A786
:104EB000DAD8FB12A7DAFC53040FC4540F75F00ABA
:104EC000A42CFC249C50027C0078D78601E4B92FE6
:104ED00002D2E72CF6786412A7DAF608B86AF8125C
:104EE000A7DAE5386003024E5412A7DA12A7DAC235
:104EF000ACC322907EA88003907EBA7F207E0012F1
:104F00004CF512A88702A9B7753400C26B124FC0C6
:104F100012A9B7125332E5166003124F20020200A5
:104F200012557A12109312A88710002010010280E7
:104F3000F8125381501312109E124EF310000D10F0
:024F400001026C
:104F420080F812103780D712512222C26BD22775F5
:104F5200480A121D63753400125450753703C26A31
:104F62001225F5106A051201F180EA1201F11252BE
:104F7200C412540012545C12557A12109312A8876C
:104F820010003810010280F8125381501BE9651598
:104F9200601812109E124EF312A9AF10001D1001DC
:104FA2000280F812103780C3D26B12542C75160788
:104FB200855917121DDC753500809A0202001253C2
:104FC20032124FE012545C7F19124FFA7E12907E19
:104FD200E6124CF57E23E516129F2B02A887786213
:104FE200E4124FF178D0745F124FF118E4F6227F89
:104FF20008F608DFFC227F7B7E0078107420129F67
:105002008DCE2404FED8F5227F197E08124CF57E3F
:105012002890825730530390825C024CF5C26B1287
:105022004FE012502A020200C25112545C907EDEFE
:1050320012500A1210661253327F20124FCB12A85E
:1050420087E516700512A9AC803675A6FF305103AC
:10505200124D751233EED2AC200025306DFA124E8D
:105062005B400C1253814011125122D25180BB106D
:105072005003124EF8C25180D1D251124EF380CA5F
:10508200C2AC22D22775480A121D63753400C26B66
:10509200125450753703C26A1225F5106A051201BF
:1050A200F180E81201F11252C412540012545C123F
:0250B20050B9F3
:1050B40050D70202009082FF12500A12107812A8F0
:1050C40087C310001310010510020E80F4124DD096
:1050D400400122124EF880DDD3C2AC22D227C26B2B
:1050E40075480A121D63753400125450753703C293
:1050F4006A1225F5106A051201F180EAD26B125288
:10510400C41254001252EC75B901E5BCB2E7F5BC07
:105114001239E4751607855917121DDC80C8D26B45
:1051240012542C125303E51775F01084240AF54821
:1051340024E8500375480A121D6F85585922D2205D
:10514400753200128CB675A704900700751500120D
:1051540052EC75B901E5BC20E705E515F0800C04B7
:10516400600975BCFF75B90575B9020515E5152407
:105174002050DCE58224FE4003025219A882187FE5
:105184000075A7007583078882E0FE75F004A412F9
:105194005297A9BCAABDABBEACBF1582E0FD75F0A9
:1051A40004A4125297C3E995BC404C7052EA95BDD1
:1051B4004045704BEB95BE403E7044EC95BF403784
:1051C400703DEE75F004A404125297A9BCAABDABBD
:1051D400BEACBFED75F004A404125297C3E995BCAC
:1051E4004015701BEA95BD400E7014EB95BE400748
:0351F400700DEC4F
:1051F70095BF5008EEF00582EDF01582E582600953
:10520700C3EF9582500302518D0FC3E89F400302FD
:10521700518575A70490070075C70375C6A8E0F503
:10522700BCE0F5BDE0F5BEE0F5BF75B90575B9029F
:1052370005C6E58224204006E5C6242050E008750F
:10524700C70375C68075B901E5BC125281F5BCE587
:10525700BD125281F5BDE5BE125281F5BEE5BF1202
:105267005281F5BF75B90205C6E5C6245850D6E583
:10527700320470FB75A700C22022B4FF0122F97522
:10528700A704900700E582686005E06970F7E922E6
:10529700F5C685F0C775B901E5BC645F700375BCD9
:1052A70027E5BD645F700375BD27E5BE645F7003C6
:1052B70075BE27E5BF645F700375BF272275C703F7
:1052C700E54875F004A42480F5C6E55975F0048413
:1052D700A8F00825C6F5C675B901A9BCAABDABBE1D
:1052E700ACBF861522E515242050037515DFE5159B
:1052F70075F004A454FCF5C685F0C722E5172420F1
:105307004028E51775F00484A8F00824A8F5C675A9
:0F531700C70375B901A9BCAABDABBEACBFA61533
:1053260089BC8ABD8BBE8CBF1239E422E4F516F522
:105336001579FF1252EC75B901E5BCB4FF040516E8
:10534600A9150515E515242050E9891579FF75C7B6
:105356000375C6A875B90109E5BC04601B09E5BD5E
:1053660004601509E5BE04600F09E5BF0460090580
:10537600C6E5C6242050DD098917227900E975F0B3
:1053860004A454FCF5C685F0C775B901E5BC20E751
:105396003078D066702B08E5BD66702508E5BE66D8
:1053A600701F08E5BF66701905C675B90108E5BC2A
:1053B60066700E08E5BD66700808E5BE667002D325
:1053C6002209E9242050B6C3221253EF1253D7A85C
:1053D600017F08E0F608DFFB221253EF1253E7A81D
:1053E600017F08E6F008DFFB2278D0796275A70412
:1053F600758307EBC454F0F582221252EC78D01272
:10540600541AE5BCF9C23C20E702D23C12541A7881
:105416006212541A75B901A6BC08A6BD08A6BE0834
:10542600A6BF0805C622D2201252EC78D012543EEE
:0554360012543E7862F3
:10543B0012543E86BC0886BD0886BE0886BF08127D
:10544B0039E405C6221244C412AA5A12668402A871
:10545B008712AA5A7F007E09907ECB124CC47F0A1A
:10546B007E12E51504129E637F1412979E1210375D
:10547B007F277E0875130778D0124D40E6793E30B2
:10548B00E702792F7E34E9129FBF7F3D7E01907F2B
:10549B0003124CF520311B303003125A96C23B12CB
:1054AB00570C1254C2D23B12570C1254D4125753EE
:1054BB00807C128E9080E6C23B7F4474532017028F
:1054CB00744E7E00129FBF8017D23B7F4F745720C4
:1054DB00170274457E00129FBF7E06E51E129FAC1D
:1054EB007E0CE51D129FAC7E12E51C129FAC7E1745
:1054FB007464129FBF7E1CE51B129FAC7E22E51AC3
:10550B00129FAC7E28742E3026027427129FBF7E0A
:10551B002DE519129FAC7E33E518129FAC7E393006
:10552B002607742C129FBB7E3BE537029FAC742D74
:10553B00201702742B7F707E15129FBF1255577E5A
:10554B003A129E0C7E01907F2F024CC47E1BE51CF1
:10555B00129FAC7E21E51B129FAC7E27E51A129F92
:10556B00AC7E2DE519129FAC7E33E518029FAC1271
:10557B0055F81256231258FA12545C12595420172C
:10558B001E10021B12347B1295FC1255E0121046B2
:07559B007F347E2F124D5AF0
:1055A20012549512A88780E212103720302620313B
:1055B20028C23B12570C125638786612580CD23B4E
:1055C20012570C12564D786912580C125753125634
:1055D200C70258AF125B6180F2128EA580EDE57DA5
:1055E20075F01084AAF075F00AA42A547FFA78D7CD
:1055F200E654802AF6227F277E0879D08700C001F0
:10560200D224B9D002C2241259DBD001A700102340
:105612000909EE2406FEB9D7E32219EE24FAFE8028
:10562200DB7E3479D7E7A2E7921712598879D7E758
:10563200A21792E7F722C224C23B751E007F447E66
:1056420000125998801E1023ED802AD23BC2247F7B
:105652004F7E001259A0D2247E06E51E1259CDF5C6
:105662001E1023E7D2247E0CE51D1259CDF51D3004
:105672003BD41023E1D2247E12E51C1259CDF51C35
:105682001023E17E1CE51B1259CDF51B1023E67E8B
:1056920022E51A1259CDF51A1023E87E2DE51912CA
:1056A20059CDF5191023E87E33E5181259CDF518B6
:1056B2001023E87E393026027E3BE5371259CDF5BC
:1056C200371023E3227F707E15125990C2247E1B6D
:1056D200E51C1259CDF51CD2247E21E51B1259CDB1
:0956E200F51B1023E77E27E51AF1
:1056EB001259CDF51A1023E67E2DE5191259CDF579
:1056FB00191023E87E33E5181259CDF5181023E85D
:10570B002278D7E6C2E775F00A847866F537303B26
:10571B0005786985F03712577C30262BE53775F005
:10572B0003A4040475F00584FBE51975F00AA425A0
:10573B001875F006A42BFBE435F0FC123E83F5370D
:10574B00123E83F5188B1922E563FC339217AB627B
:10575B005003123EF4305C0A7AD2123C6F7840123E
:10576B003E11AE04AF037C277D10123D7A8F1C8057
:10577B0037E6FD3392171886041886035003123E42
:10578B00FC7A09792778C0123E0E8B1EADD3ACD2B2
:10579B00AB0679EA7860123E0C8B1DAF06AED27C5D
:1057AB00177D70123D7A8F1CAF05AE047C037DE82C
:1057BB00123D7A8F1BAF05AE047C007D64123D7ADF
:1057CB008F1AED75F00A84F51985F01822EC3392D7
:1057DB00175003123EF4751D30301786751D2D8042
:1057EB008178427B607CEA800678407B207C4E127D
:1057FB008F7079277810123E0C8B1CAF06AED280BF
:10580B00AB30262AE51975F00AA4251875F00AA401
:04581B002537FBE44E
:10581F0035F0FC7A05123C618C068B077C007D030A
:10582F00123D6D8E048F03125746E51E75F00AA4C4
:10583F00251D75F00AA4251C75F006A4251BFBE495
:10584F0035F0FC7A0A123C61EB251AFBE43CFC7A3A
:10585F000A123C6FEB2519FBE43CFCE43DFD7A0A90
:10586F00123C81EB2518FBE43CFCE43DFD301703B3
:10587F00123EFCA60518A60418A60378D7E6A2E7E1
:10588F00923DC2E775F00A84FCABF0303B0EAB37AC
:10589F00EC75F00AA42BA23D92E7F622AC3780F00C
:1058AF001258CA305C0A7A40123C6F78D2123E11FD
:1058BF00301703123EF48C638B62221258DA7A0A85
:1058CF00123C61EB2518FBE43CFC22E51C75F00A49
:1058DF00A4251B75F00AA4251AFBE435F0FC7A0AFF
:1058EF00123C61EB2519FBE43CFC2212592C12A946
:1058FF00B3C202C22312592C100008100105100266
:10590F001B80F51031ED10300D102604D22680E3E8
:10591F00D230C23180DDD231C23080D7227F357E86
:07592F0000907EEC124CF524
:10593600907F0A20300F907F1A203109907EFB203D
:105946002603907EF31F7E17124CC402A8877F356C
:105956007E01907F22124CF57F347E3A125A7D7476
:105966004E129FBF12A88712A9B3C2027F347E3A95
:10597600D21775115975124E802675112E7512277C
:10598600801E75113E75122F801675112B75122DFE
:10599600800E75114E751253800675114575125796
:1059A600125A7DE511301702E512129FBF12A88721
:1059B60010000810010510020B80F5D23C1017E309
:1059C600D21780DF025A784430F81259D7E8540FBC
:1059D60022C2218002D221A22492229223125A7D2F
:1059E600E830E709D23C7430302102745FF8129F28
:1059F600BF12A88710003410010510025D80F5D291
:105A06003C102266102367B43909745F2021DF74C5
:105A16003080DBB45F04742D80D4B42D04744180CF
:105A2600CDB45A04743080C60480C3D23C302406F8
:105A3600102237102338B44104742D80B1B42D04DC
:105A4600745F80AAB45F04743980A3B43009745AB1
:105A560020219B74398097148094B47108D223E86E
:105A6600129FBF800DF8C223800874718001E8027E
:105A760059F4905A928003905A8EC007EF2408FF7B
:105A8600129FEDD00702A8870205F8F8020500006C
:10A8270075A70090A85975F02D84C2D5C2D16017BD
:10A83700D2D1146007D2D514600DC2D1E5F093FCD4
:10A84700742D95F093FB22E5F093FB742D95F0930F
:10A85700FC220009121B242C353E474F58606870B4
:10A867007880888F969DA4ABB2B8BEC4CACFD4D91E
:10A87700DEE2E6EAEDF0F3F6F8FAFCFDFEFFFFFF95
:10A8CC00D23D8002C23DED8BF0A430E70205F0C30F
:10A8DC00E895F020D50425F025F0FEED8CF0A430A1
:10A8EC00E70205F0C3E995F030D10425F025F0FF1F
:10A8FC00203D0B2487500122EF24CC40012202A9D9
:01A90C004CFE
:10A61500203A437E1C7F5312A94C7F5912A94C1E28
:10A625007F5712A94C7F5512A94C7E2312A94C7F46
:10A635005712A94C1E7F5912A94C7F5312A94C1FC2
:10A645007E2012A94C7F5A12A94C7E1E12A94C7F5E
:10A655005212A94C800A7E1C7F5390A69B129FED37
:10A6650030741CE5716018E57012A827781F7956BB
:10A675007D0912A8D0303A0312A6850DBD16F32226
:10A68500C0060E30D5021E1E12A94CD0061F30D1B1
:0FA69500020F0F02A94C070700386C446C380005
:1096210030122D907F397F717E2F124CF5128CA252
:109631007A0AC23D129862203D16DAF81297647CCC
:10964100007D03123D6DEFA2D17E237F6512A084C0
:10965100227F567E051297AA7F3D1297BD7F6F121A
:1096610097BD7E1F7F411297FA7E0A7F4112981C97
:109671007E227F5912981C20120122128CA2857A17
:109681001D855E1C857B1B855F1A7AC0C23D1298C1
:1096910062BAB7048C1C8D1D203D521297647C0068
:1096A1007D14123D6D74562F20D1029F9FFF24CB54
:1096B10040028037EF248850028030EA1475F003AD
:1096C10084FE12A94CC3E51B957BFEE51A955F92BA
:1096D100D55004EEF404FEEEC313FE24E0400C74F6
:1096E1001F2E30D5029E9EFE12A94CDAA120120136
:1096F10022AC1CAD1D1297647C007D03123D6DEF01
:10970100A2D17E047F5392D175F080305C04F5F0D4
:109711008001A4A2E792D5E5F075F03284F8E5F076
:1097210075F00584C0E0E5F0A2D533C0E0E860271C
:10973100129FA5EE2406FED0E0F8D0E0129FA5EE20
:0A9741002405FE742C129FBF0E0ECB
:10974B00E8129FA57E007F547420029F8D742B20FE
:10975B00D102742D129FBF80D0C3ED957AFFEC958B
:10976B005EFE92D15003123EE422128CA2857A1D2A
:10977B00855E1C7A0AC23D129862203D06DAF88C8F
:10978B001C8D1D227F151297967F327E3E12A94C9F
:10979B00DEFB227E0E12A94C0EBE31F9227E011287
:1097AB00A94C0E0EBE3FF8227E3312A94C0EBE40C2
:1097BB00F9227E047D1112A94C0E0E0EDDF81F1F2F
:1097CB007E35907F3D305C057E31907F41024CF5BC
:1097DB007405305C097E327401129F7A74067E36F2
:1097EB00129F7A7E3A7400129F7A7E3D029F7A7D99
:1097FB000F12A94C0F0F0FDDF8227F737D0380042E
:10980B007F727D0512A94C0FDDFA227F717D0780D7
:10981B00F37D0A12A94C0E0E0F0FDDF722203D0728
:10982B00122BC67003D23D22056D128ACAE4F5F7DE
:10983B00C2B2C2B2ABF7F5F7C2B2C2B2E5F7FA30B9
:10984B00E411EB251DF51DE4351CF51C0519EA305B
:10985B00E3010ED2B280117803203D07122BC670A4
:0A986B0003D23D22D8F3056DE56D30
:109875002409F56D128ACAE4F5F7C2B2C2B2ADF792
:10988500F5F7C2B2C2B285F71BF5F7C2B2C2B2E5AF
:10989500F7FCD2B2C220543F30E50244C0CC54C0DC
:0B98A5002323F51AE56D24F6F56D2273
:10A583007E017F0990A601129FED2051097E037F72
:10A5930000743F029FBFE4FEFFC3E545129B3DFDF0
:10A5A300940AED403D9464ED40027463129E5D7E17
:10A5B300017F09E552240575F02D84AAF075F00595
:10A5C300A4CA75F00B842A90A5EC9312A827BCB8F3
:10A5D300027BB87D04EE2DF8EF2DF90D12A8CCDD2A
:10A5E300FB227E03129FAC80C6000C1622222D395B
:10A5F300444F4F5A66707C7C87939EA9A900090932
:10A6030008004100000000008880000000004100B5
:02A6130008003D
:109B3D00305D0A75F08AA42480E5F03400227F00A0
:109B4D002074147E110F909BD7129FED7F0A7E0A11
:109B5D00E52E5407029E747E0BE571B4FF2DE55181
:109B6D0024025003755100E551129B3D75F005A47B
:109B7D00ACF0FB123C377E0D781CE66004E6129FBC
:109B8D00A5EE2405FE18B818F48006129B3D129E12
:109B9D00637F0C7E11E571602B0EE57064B460245B
:109BAD0064B475F03284C0F0129FA5CE2405CED0DA
:109BBD00E075F00584C0F0129FA5CE2405CED0E04F
:109BCD0023029FA59067E5024CC4070FFFFF9EE798
:109BDD00AD6B9C6BAD6B9D67FFFF75548030745DF5
:109BED0078BD79BBE6FC27FB1819E6FD37F9EBF8D4
:109BFD007B00123E138B547F087E11A806909C4B60
:109C0D00129FED30100F20730C7F0A7E1712A97C66
:109C1D000E0E12A97CE5542483E554500224FA75E6
:109C2D00F01984FB909C539328FEEB909C5D93FD63
:109C3D0012A94C0F0F12A94C1F1F0EDDF322030F9B
:109C4D000100FFFE03800000000007070D0C0B0A4A
:109C5D0005040302010102030405E57E7001227F64
:109C6D00357E00746F129FBF7E06E57E129B3D020E
:109C7D009ECE202C0122909C89029FED050EFFF0B7
:0C9C8D00E01CF004F81CFFF03012012273
:109C99007F151297967F1F1297967F291297967FA5
:109CA900177E06E53F30E00B907F5D305C03907FC7
:109CB9007180132074077E01907F468009907F523E
:109CC900305D03907F67124CC4307306E53960023A
:109CD900153920571BE539B4011612064C128A6A48
:109CE900C3E55C9560F5BCE55D9561F5BD1239E4A8
:109CF9007F217E01E53F30E01E305705907F7B8054
:109D090020E5397005907F878017907FA9124CC490
:109D19007E30E539029EC8302B0AE5397007907FFD
:0A9D290092124CC422907F9D80E34B
:109D3300123C097F207E05751900781DC2D5E630D7
:109D4300D517129FA5EE2405FE18B818F17E1F74CF
:109D530063305C027465029FBF7005B8191880E216
:109D6300D2D5CE24FACE746B301702742D129FBF56
:109D7300EE2406FE80C87420129FBB80C87F007E3D
:109D830023AC5EAB7A123C09781DC2D5E630D50C04
:109D9300129FACEE2406FE18B818F1227005B8190C
:109DA3001680EDD2D53017E4CE24FACE742D129F4F
:109DB300BFEE2406FE80D57420129FBF80D5123CCF
:109DC30009781DC2D5E630D516129F7AEE2404FE1B
:109DD30018B818F10E745E305C027427029F897004
:109DE30005B8191680E3D2D53017DACE24FCCE7429
:109DF3002D129F8DEE2404FE80CB7420129F8D8044
:109E0300CBC23D129E170F0F0E0E7463305C0274AB
:109E130065029FBF123C09781DC2D5E630D50C12EE
:109E23009FDCEE2408FE18B818F1227005B8191645
:109E330080EDD2D5301716740BCE24F8CE129FDCEA
:109E4300EE2408FE80D5740C129FDC80D5303DCB08
:049E5300740A80E528
:10A225007F797E24E55F30E70122AC5F1CAB7B12B2
:10A235003C37E51B700E7420129FBFEE2405FE12FD
:10A24500A273800C12A273E51B129FA5EE2405FED6
:10A25500E51A129FA5EE2405FE742C129FBF0E0E63
:10A26500E519129FA5EE2405FE745E029FBF742DAD
:10A27500201702742B129FBFEE2406FE22E55F30E5
:10A28500E70122AC5F1CAB7B123C37E51B700E74FB
:10A2950020129F8DEE2404FE12A2CC800C12A2CCBB
:10A2A500E51B129F7AEE2404FEE51A129F7AEE242E
:10A2B50004FE742C129F8D0E0EE519129F7AEE2462
:10A2C50004FE742A029F8D742D201702742B129F91
:06A2D5008DEE2404FE22C0
:10A07C007E257F09A275E579C23D6002D23D92D161
:10A08C0075F080305C04F5F08001A4A2E792D5E570
:10A09C00F075F03284F8E5F075F00584C0E0E5F079
:10A0AC00A2D533C0E0E86027129FDCEE2408FED076
:10A0BC00E0F8D0E0129FDCEE2408FE0F0F205A1FB0
:10A0CC007460129FBF1F1FEE2404FEE8029FDC7415
:10A0DC000C303D06740A20D10104129FDC80CC2088
:10A0EC005904742E80DC205804746180D57462800D
:10A0FC00D1A275E579C23D6002D23D92D175F08056
:10A10C00305C04F5F08001A4A2E792D5E5F075F07F
:10A11C003284F8E5F075F00584C0E0E5F0A2D533A3
:10A12C00C0E07F3E7E1CE8602012A03DD0E0F8D05D
:10A13C00E07F3E7E2812A03D7F447E32742E129F1B
:10A14C00BF7F3E7E37E802A03D303DE0740A20D14F
:07A15C00010412A03D80D5B3
:1098B000E54424F64001227800E5520475F0038463
:1098C000F9E928FE24C45001FE1298E81298F41E0B
:1098D00012A94CC3E998FE5003243CFE1298E81EDE
:1098E00012A94C08B81FDA22EE2420FE24C250032D
:1098F0002402FE22E824F1E8C2D55006D2D5E8F4CD
:10990000241F23FF90997293CF0493FAE545F5F055
:10991000A4ACF0FB123C98E544F5F0A49BFBE5F009
:109920009CFCEB2420FBEC3400FC24F0500CEB24DA
:1099300060EC34009099C293800EEB33FBEC33FC67
:10994000EB33EC3390999293FAE5458FF0A430E72E
:109950000205F0E5F020D502F4042A75F00520197F
:109960000375F00384FF24DF50027F20C374329F0D
:10997000FF22FF00FF03FA0BF318EA2ADE40CF585C
:10998000BE73AB8D96A880C068D64FE835F51BFD39
:1099900000FF00080B0E101214151718191B1C1DC0
:1099A0001E1F20212223242526262728292A2A2B68
:1099B0002C2D2D2E2F2F3031313233333434353698
:1099C0003637373839393A3A3B3B3C3C3D3D3E3EF1
:1099D0003F3F4042444648494B4D4E5052535556E6
:1099E00058595B5C5D5F60616364656668696A6B5A
:1099F0006D6E6F7071727374767778797A7B7C7D17
:109A00007E7F808182838485868788898A8B8B8C00
:109A10008D8E8F9091929394949596979899999A08
:109A20009B9C9D9E9E9FA0A1A2A2A3A4A5A6A6A723
:109A3000A8A9A9AAABACACADAEAFAFB0B1B1B2B34F
:109A4000B4B4B5B6B6B7B8B9B9BABBBBBCBDBDBE88
:109A5000BFBFC0C1C1C2C3C3C4C5C5C6C7C7C8C8CC
:109A6000C9CACACBCCCCCDCECECFCFD0D1D1D2D219
:109A7000D3D4D4D5D5D6D7D7D8D8D9DADADBDBDC6E
:109A8000DDDDDEDEDFDFE0E1E1E2E2E3E3E4E5E5C8
:109A9000E6E6E7E7E8E8E9EAEAEBEBECECEDEDEE29
:109AA000EEEFEFF0F1F1F2F2F3F3F4F4F5F5F6F690
:109AB000F7F7F8F8F9F9FAFAFBFBFCFCFDFDFEFEFE
:109AC000FFFFE54524FD400122E5520475F00384C3
:109AD000241FFE24C250032402FE129B13EEFD2419
:109AE0001EFE24C250032402FE129B13E5442402EE
:109AF00075F00520190375F00384F4042432FF2463
:109B0000EE500F129B08AE051E1E7C0512A94C0ECE
:109B1000DCFA227F1512A94C0F0FBF2DF822E55356
:109B20000475F00384241FFE24C250032402FE1295
:0D9B30009B330E7F2312A94C0FBF2DF9228D
:10A163007E3974373019027455129F15801C75A7F8
:10A17300007E007F2F90A200129FED205DE27E35CE
:10A18300746430190274A0129F2B30745A30125722
:10A19300E54AB4040122B4060122E57112995BEF8A
:10A1A300FDE5700475F00384241EFE24C2401F24C1
:10A1B30003501E90A1EB600990A1F214600390A1DB
:10A1C300F9E493A3B4FF0122FE12A1DF80F324027A
:10A1D300FE7C04EDFF12A1DF0EDCF822EDFF12A9D5
:10A1E3004C0FEF24CE50F7223B3C3D3E0001FF3C99
:10A1F3003D3E010203FF3E3F01020304FF053870A9
:10A2030001100240078080011003400400600150E8
:10A2130003C0070017FCA7FADFF43FE000A00240E9
:02A223000780B2
:10A9FF00AF177E00E53C129E577E0C742E129FBF40
:10AA0F007E12E53B129E577E1E742E129FBF7E2430
:05AA1F00E53A029E571C
:10A90D007F797E16743B129FBB7E18E53F129EC267
:10A91D007F797E0078AEE6129EC27E0A743B129F4E
:10A92D00BB7E0CE53E029EC27F797E00E540129E05
:0FA93D00C27E0A743B129FBB7E0CE541029EC294
:10A43C00751700787512A48F7453201702744E2070
:10A44C007406E52E54074430AF1712A4B97E3BE5D1
:10A45C007DC4540F129FAC2074077E077420129F8A
:10A46C00BF787812A48FE5172409FF7457201702C0
:10A47C007445207402742012A4B97E3BE57D540F00
:10A48C00029FACE6FD33921718860418860330172A
:10A49C0003123EFC79177870123E0C8B13AF06AE8C
:10A4AC00D27C007D64123D7A8F148D15227E0012B1
:10A4BC009FBF7E07E513129E747E197464129FBFB2
:10A4CC007E20E514129E577E2B742E2073030E747F
:0BA4DC002C129FBF7E2FE515029E573B
:10A38E00C234E54A603B7A2420E00E7A261414602B
:10A39E00087A28141460027A297F717E00303F0AF1
:10A3AE00E537640260047F6B7E05EA129FBF20557D
:10A3BE0005205406800B745B8002745C7E00129F35
:10A3CE00BF30262EC2267F687E0090A415124CC484
:10A3DE007F66A85AE54AB4060108E875F0648474ED
:10A3EE000AC5F084C0F0129FDCEE2409FED0E01204
:10A3FE009FDC200811E537B402032041097F367E29
:10A40E002E7441129F8D224D41524B00E54375F043
:10A41E0008A495355011E59020E20CD2347E237FAE
:0EA42E007190A436124CC422455849543F0088
:10A2DB0020144F740512AA44EF33EE33F9EF030346
:10A2EB00541FF5F090A32EE993A4C5F013C5F013FA
:10A2FB00C5F013C5F013C5F0135403FCE5F013FBC5
:10A30B00E9242093C9244093C39BC4540FFBE99CBD
:10A31B00C4FC540FF9EC54F02B2446F57BE934F6CE
:10A32B00F55F22FFFFFFFFFFE6C5AD9C8F857D77B5
:10A33B00726E6C6A696A6A6C6F747A828D9DB4D91D
:10A34B00FFFFFFFAE9DCD3CEC9C6C3C0BEBBB9B7AA
:10A35B00B5B4B2B0AFADABAAA8A6A4A2A09E9C996F
:10A36B0096918C00381CE735D137246F00C5B3C1EB
:10A37B00E61F66B60E68C21867AADBF4EDB9467520
:03A38B0010A2001D
:10AA2400D2A27408D2A1D2A300C2A3C2A1D2A3000D
:10AA3400C2A3D5E0EF7405D2A300C2A3D5E0F822E7
:10A9D800C2A3D2A2D2A1D2A300C2A375F008339217
:10A9E800A1D2A300C2A3D5F0F5C2A175F003D2A3EA
:07A9F80000C2A3D5F0F82214
:1092790012A9D8D2A300C2A3C2A175F008E4D2A34F
:1092890000C2A3A2A233D5F0F5FE75F008E4D2A37B
:1092990000C2A3A2A233D5F0F5FFD2A300C2A32234
:1092A900E478806608B88BFB70012274D512927934
:1092B9007881C3EE13FEEF13F692D118EE2460F60F
:1092C90074D61292797888EF33CE33CE33CE33CE3B
:1092D90033A2D192E25407FCEEFB7A08123C61EC0E
:1092E900244FF608EBF674D9129279EF543F78823D
:1092F900F67886EF33CE33CE33CE33CE335403F6FE
:1093090008EEF618161608E6C4FF54F0F618E6C477
:10931900CF540F2FF674DA129279EF232354FC7885
:1093290083F67884EEF608EF54C0F67880E4660890
:10933900B88AFBF6221292817889C3EF96FF18EE5C
:0893490096FEA2E792165010F7
:10935100123EE4740FF8F9123CAEEF2CFFEE3DFE25
:10936100788BEEF608EFF622E6182016072CF7E6C2
:109371003D19F722C39CF7E69D80F66A405E805650
:10938100E050F04B0044803DC0384031D02BA02547
:10939100601F2018D001440158016801780188013B
:1093A100A001B401D001EC02100238026802A078D9
:1093B100BE8020858E8A9D8F4D95BA9A97A0BEA6B4
:1093C10031AC53B22AB801BD6F129281788DEEF69D
:1093D10008EFF67887798C123CAE788379901293F6
:1093E100697885798C123CAE78817992129369788B
:1093F1008DE624E4FE08E63392D13392D554FCFF86
:10940100EEA2D133A2D533FE780F7992123CAE7819
:10941100947990C3EC97F61819ED97F67994909397
:109421007C7F197D0EEF93C3971F19EF93971F0947
:109431001DED600240EF0F909396798DEF93F70940
:109441000FEF93F7788E7994123CAE9093B0EF932F
:10945100C39BFB1FEF939C2420FC7897E62BF61807
:10946100E63CF618E436F6740612AA44D237EE2426
:07947100F74006240250023F
:10947800C237EEFCEFFD740712AA44C3ED9FFFEC60
:109488009EFE78B7E6FD337C0050011CEF2DFFEE01
:109498003CFE78D8E6C4540F2FFFE43EFE789CEFDC
:1094A80026F618EE36F62220141220370F789DE69D
:1094B800B4050912954B1295801295C422201442C6
:1094C8007897799A1295DF123E6CC3EE9420FE923B
:1094D800455003123EE47C007D05123D7A30450379
:1094E800123EE48E618F6012A56975C70375C6FECA
:1094F80075B901E5BC2560F57AE5BD3561F55E1203
:10950800A5767897799AC3E697FB1819E697FC7AB7
:1095180002123C6130370B7A02123C61ECFEEBFF21
:10952800800312954B1295802014031295C47895E8
:109538007998E6F776000809E6F776000809E6F76D
:10954800760022799CE77700FB19E77700FC789D85
:10955800E6B40506EB33FBEC33FCECA2E792D550FE
:0A95680003123EF47A32123C6FEC5D
:10957200FBEDFC30D503123EF4ECFEEBFF22EE24B1
:1095820008FE7404203711789DE6B40504740C803B
:1095920007F42406C323540FFD7C00123C4D789F30
:1095A200E6FC08E6FBC374109DFA123C6FEFF8EE7E
:1095B200F9123E6CE878A02FF6FF18EE39F62480F7
:1095C200FE2292754003123EE4EF33EE33F579C288
:1095D20076307508E57924F15002D27622E627FB2F
:1095E2001819E637FC1819E637FD22128C497F0854
:1095F2007871793A12960802362B855E63857A6213
:10960200787379647F06E6F70809DFFA22786479CD
:0F9612007380F1787379AF80EB78AF797380E56F
:103BE700E4FEFFFC7D0A791DE7540F2FFFE43EFE3C
:103BF700B91902800619123C4D80ED301703123EA9
:103C0700E422305C2BEC3392175003123EF4EC2481
:103C1700D950047C277B007AD2123C6FEB33CC332C
:103C2700CD33CC33ED33FBEC33FC301703123EF4CA
:103C3700EC3392175003123EF47919123E83F709B9
:103C4700B91DF8A70322EFF88DF0A4FFEDC5F0CE5C
:103C5700A42EFEEC88F0A42EFE22EB8AF0A4FBE54E
:103C6700F0CC8AF0A42CFC22EB8AF0A4FBE5F0CC84
:103C77008AF0A42CFCE435F0FD22EB8AF0A4FBE5E6
:103C8700F0CC8AF0A42CFCE435F0CD8AF0A42DFD0D
:103C970022EB8AF0A430E70205F0E5F0CC8AF0A425
:103CA7002CFBE435F0FC2286F0E7FDA4FAABF01913
:063CB700E786F0A42BFBE0
:103CBD00E435F0FC18E68DF0A42BFBEC35F0FCE4BC
:103CCD0033FDE687F0A42CFCED35F0FD22EB89F0F9
:103CDD00A4CBAEF08AF0A42EFEE5F03400FDEC8905
:103CED00F0A42EFEE5F03DFDE433CC8AF0A42DFDCD
:103CFD00E5F03CCEFC22EB89F0A4CBAFF08AF0A42A
:103D0D002FFFE5F03400FEEC89F0A42FFFE5F03E27
:103D1D00FEE433CC8AF0A42EFEE5F03CFCED89F0F8
:103D2D00A42EFEE5F03CFCE433CD8AF0A42CFCE59A
:103D3D00F03D8E058C068F04FF22C2D5EC30E705D1
:103D4D00B2D5123EECEE30E70DB2D5123EE4123D87
:103D5D007A123EEC8003123D7A30D503123EE422F6
:103D6D00C3EC13C0E0ED132FFFD0E03EFEBC000B03
:103D7D00BE0029EF8DF084FFADF022E4CCF975F093
:043D8D0008EF2FFF0D
:103D9100EE33FEEC33FCEE9DEC994005FCEE9DFE0E
:103DA1000FD5F0E9E4CEFD22EDF9F5F0EE8420D255
:103DB1001CFEADF075F008EF2FFFED33FD400799C4
:103DC1005006D5F0F222C399FD0FD5F0EA22EC336B
:103DD100EE3400FEEF3400FF7D007A0079007809AF
:103DE100C3ED9AFDEE9BFEEF9CFFB392D54009ED2A
:103DF1002AFDEE3BFEEF3CFFA2D5E933F9ED33FDA1
:103E0100EE33FEEF33FFD8D92279007A00C3801553
:103E110079007A00C3EA13FFE913FEE8132BFBEEE6
:103E21003CFCEF3DFDE4F5D2F5D333FE7F19C3EE43
:103E310098FEE5D299F5D2E5D39AF5D3B392D54060
:103E41000DEE28FEE5D239F5D2E5D33AF5D3A2D568
:023E5100EB3351
:103E5300FBEC33FCED33FDDF0122EE33FEE5D23321
:103E6300F5D2E5D333F5D380C3EDC454F0FEECC4EF
:103E7300FF540F2EFEEF54F0FFEBC4540F2FFF221D
:103E8300EC75F00A84FCEB54F025F0C475F00A8459
:103E9300C4CBC454F025F0C475F00A842BFBE5F0C1
:103EA30022AC10AB11123E83A904AD03FA7C197B3B
:103EB30099123C61AE04AF03EA75F006A4F8AC12A4
:103EC300AB13123E832875F00A8485F014F8EF2BA8
:103ED300FFEE3CFEEF28FFE43EFEE43DFDE439FC4B
:103EE30022C3E49FFFE49EFE22E4C39DFDE49CFC09
:103EF30022C3E49BFBE49CFC22C3E49BFBE49CFC09
:103F0300E49DFD2275D4107B807A0079807800EAE5
:0A3F1300F5F0A4FCADF0EBF5F0A40E
:103F1D00FEAFF0EB8AF0A4C333C5F033C5F092D5F4
:103F2D002DFDC5F03EFEE430D501043FFFB5150D66
:103F3D00EEB51409EDB51305ECB51201224006EAF4
:103F4D0098FAEB99FBD5D40ABB0001220ABA0001FD
:103F5D000B22C3E913F9E813F8EA28FAEB39FB80D1
:103F6D00A478087B807D807C00EDF5F0A4FAE5F067
:103F7D008EF0B5F007EA8FF0B5F001224003ED9B0E
:103F8D00FDD827BDFF0122EDF5F0A4F9A8F0ED0451
:103F9D00F5F0A4C399FAE5F09813CA1329F9E83A94
:103FAD00F8C3E99FE89E50010D22C3EB13FBED2BE7
:103FBD00FD80B67473F8F9123FD47547FFEF20E119
:103FCD000513EE13F54722E627FA0809E637FB0835
:0E3FDD0009E637FC30E70AC3E49AFAE49BFBDE
:103FEB00E49CFCEA75F01FA4AAF0EB75F01FA42A61
:103FFB00E5F03400FBEC75F01FA42BFBE5F034006F
:10400B00FC90402760020583EB93FE70037F022236
:10401B007F01BC0106EB24AC50011F220000000005
:10402B0000000000000000000000FFFFFFFFFFFF8B
:10403B00FFFFFFFFFFFEFEFEFEFEFEFEFDFDFDFD94
:10404B00FDFDFCFCFCFCFCFBFBFBFBFBFAFAFAFAB0
:10405B00F9F9F9F9F8F8F8F7F7F7F7F6F6F6F5F5E1
:10406B00F5F4F4F4F3F3F3F2F2F2F1F1F0F0F0EF24
:10407B00EFEEEEEEEDEDECECEBEBEBEAEAE9E9E87B
:10408B00E8E7E7E6E6E5E5E4E4E3E3E2E2E1E1E0E5
:10409B00E0DFDEDEDDDDDCDCDBDADAD9D9D8D7D761
:1040AB00D6D5D5D4D4D3D2D2D1D0D0CFCECECDCCF1
:1040BB00CCCBCAC9C9C8C7C7C6C5C4C4C3C2C1C192
:1040CB00C0BFBEBEBDBCBBBABAB9B8B7B6B6B5B445
:1040DB00B3B2B1B1B0AFAEADACACABAAA9A8A7A609
:1040EB00A5A4A4A3A2A1A09F9E9D9C9B9A999897DF
:1040FB0097969594939291908F8E8D8C8B8A8988BD
:10410B0087868584838281807E7D7C7B7A797877B4
:10411B007675747372716F6E6D6C6B6A69686765B7
:10412B0064636261605F5E5C5B5A595857555453C8
:10413B0052514F4E4D4C4B494847464543424140E7
:10414B003F3D3C3B3A38373635333231302E2D2C10
:10415B002A29282725242321201F1D1C1B1A181749
:10416B0016141312100F0E0C0B0A0807060403018A
:10417B00FFFEFDFCFBF9F8F7F5F4F2F1F0EEEDEBD9
:10418B00EAE9E7E6E4E3E2E0DFDDDCDAD9D8D6D52D
:10419B00D3D2D0CFCECCCBC9C8C6C5C3C2C1BFBE8C
:1041AB00BCBBB9B8B6B5B3B2B0AFADACAAA9A7A6F4
:1041BB00A4A3A1A09F9D9C9A9997959492918F8E61
:1041CB008C8B898886858382807F7D7C7A797776D4
:1041DB007473716F6E6C6B696866656362605E5D4C
:1041EB005B5A5857555452514F4D4C4A49474644C8
:1041FB0043413F3E3C3B393836343331302E2D2B47
:10420B00292826252322201E1D1B1A1817151312C9
:10421B00100F0D0C0A08070504020101C21DC23262
:10422B00752C00C3E5679576FBE5689577FCE5692A
:10423B009578FD30E705D261123EFC24F050031255
:10424B004303AA07A906123D03EC2401FCED34003D
:10425B00FDEE3400136002D232ED13FAF519EC13B4
:10426B00FBF9F51AAC02123CDA8B128C138D148EFF
:10427B0015C3E5649573FBE5659574FCE56695756B
:10428B00FD30E705D262123EFCEBF9F51FECFAF5B7
:10429B001DED6002D23230320122123CDAEB2512D4
:1042AB00F512EC3513F513ED3514F514EE3515F554
:1042BB001540E1023F0712422720323BEB242E40F0
:1042CB00D3EA2401CB3400FC7A07793D123CDAC0E7
:1042DB0010C0118E108D118C128B13E4FCFD7E0718
:0542EB007FD0127E17D8
:1042F000851203851302D011D010BB0005BA00024D
:10430000D21D22B261C374809BFB74F59CFC7420A7
:104310009DFD22303F647F747E011297AA7E1F129A
:10432000981675A7009004EDE0A2E792171392E7A4
:10433000FC1582E013FB301703123EF4BC003BEB8C
:10434000603820E73520E63210E513201707C374E4
:104350001F9BFE80027E1F12980B0EDBFA22FB20B1
:1043600017097E00C374209BFB8008EB241FFE749A
:10437000209BFB1298050EDBFA222212961575A7D8
:1043800000758307E559C4440FF582E0A2E7925215
:10439000C2E775F00A84FEAFF075A7045382F17886
:1043A00064124400AE07786712440075A700E57DEB
:1043B000C4540FFEE57D540FFF78731243F4AE072B
:1043C00078761243F478AF79AF123FD41242C1121B
:1043D000063DA9BDE5597002A9BCE975F00AA4F92A
:1043E000EA999004ECF0A3EB95F0F0A2E7923DD2AD
:1043F0003F02961B86030886040886051818800667
:06440000E0FBE0FCE0FD22
:104406007A0A123C8120E70CEB2EF608E43CF6080B
:10441600E43DF622C3EB9EF608EC9400F608ED9414
:1044260000F622C23F302A0578A8760022E5482405
:10443600F640F9E5580460F475A700758307E55959
:10444600C42408F582E070E40582E0FFE54A6404CE
:104456006008E54A64066002801075390AEF20E7B5
:104466000975390520E603753902EF24C3400C208F
:104476003809D23878C5A64675460012063DA9BD4C
:10448600E5597002A9BCE9240DC39F401E12437B67
:10449600303D18753901204006D24078A876232091
:1044A600521BE55965586015D2332230330F055932
:1044B60078C58646C233C238C240126F3422E558E8
:1044C600B4FF012285581175A704758307E54824B2
:1044D600F65002805C201259202905202A028051BC
:1044E600129615E4F516F517751000124550E510ED
:1044F600700312960F124569302910E51B2517F532
:1045060017F51BE51C3516F516F51C1245741296A3
:104516000F0510C3E511951050D175A70002961B23
:0B452600E55AF51124F6500375110A48
:1045310075A704758306751000124550124569125E
:1045410045740510C3E511951050EE75A70022E5DD
:1045510010C4F582E0E0F564E0F565E0F566E0F5AC
:1045610067E0F568E0F5692205A7124755122DBDF0
:1045710005A722E9F0E51CF0E51BF022E510C4F5E2
:1045810082E0F512E5822406F582E0F511E0F51CE2
:10459100E0F51B2220282DE558B4FF012275A70460
:1045A10075830785591012457DE0F513E07F7A7E0A
:1045B1003D129F8DE5137E39129F8DE5127E3512D6
:1045C1009F8D802C2012012275A704758306855BBF
:1045D1001012457DE512700B7E3A7F79745D129F52
:1045E100BF800D75F06484E5F07E397F7A129F0FEC
:1045F100E53764027008304133126DB5802EE51C39
:104601007006E51B24CD5024E51164B4601EE5114C
:1046110012A827781F79567D167A1DE53F20E00400
:104621007D187A1F12A8D00DEDB502F8751619750F
:104631001779E51C24ED402BAE1CAF1B12471F7CE4
:10464100007D32123D7AC005EFAF17AE16129EC83B
:0E465100CE2405CE742C129FBF0E0ED0E02397
:10465F00129EC2801B124716124691CE2405CE74AD
:10466F002C129FBFCE2402CEE875F00584129FA5B1
:10467F00CE2404CE7422305D027466129FBF75A7DC
:10468F000022EE243D50047EC37F4B7C017DF4124B
:10469F003D7AC004C005EF6007AF17AE16129EC873
:1046AF00D007D0067C007D32123D7AA805EFAF17F8
:1046BF00AE16CE240ACE029FA5124716EE24503016
:1046CF005D03EE24A150047EC37F4B7C017DF41269
:1046DF003D7AC004C005EF6007AF177E2F129F15FC
:1046EF00D007D0067C007D32123D7AC005EFAF17A0
:1046FF007E37129F7A7E3B742C129F8D7E3DD0E0C9
:10470F0075F00584029F7AE51B2402FFE4351CFE39
:10471F00305D1ABEC305BF4D028012AC06AB077ADF
:10472F001B123C6F7832123E11AE04AF0322787326
:10473F007964123FD41242C1751CC3751B4B2032D2
:10474F00048B1C8A1B2212473D30320122AC19AE5A
:10475F001AA91DAF1FB90005BC00028010C3E913D1
:10476F00F9EF13FFC3EC13FCEE13FE80E8BF290033
:09477F005006BE2900500122C3BE
:10478800EF13FFC3EE13FE80EB3E7FE3E3E3E3E3C7
:10479800E3E3E3E3E37F3E0C1C3C7C7C1C1C1C1C19
:1047A8001C1C1C7F7F3E7FE3E3E3070E1C3870E090
:1047B800E3FFFF3E7FE3E3030F0E0F03E3E3E37F33
:1047C8003E070F1F3F77E7E7FFFF0707070707FFCA
:1047D800FFE0E0E0FEFF030303E3E37F3E1E3F73D9
:1047E800E0E0E0FEFFE3E3E3E37F3EFFFFE3E30314
:1047F80003070E1C38383838383E7FE3E3E37F3E42
:104808007FE3E3E3E37F3E3E7FE3E3E3E37F3F03CE
:104818000303E77E3C000000181818FFFF1818185B
:10482800000000000000000000FFFF000000000082
:10483800003FF00000381C38F00180C1F020F0FC87
:104848000038F03FE0000000007CC6C6C6C6C6C6F9
:10485800C6C67C1838781818181818187E7CC6C66A
:104868000C183060C0C6FE7CC6C6061C0606C6C646
:104878007C0C1C3C6CCCFE0C0C0C0CFEC0C0C0FCB0
:104888000606C6C67C3C66C0C0C0FCC6C6C67CFE62
:10489800C6C6060C18303030307CC6C6C67CC6C6C4
:1048A800C6C67C7CC6C6C67E060606CC780000183E
:1048B800187E7E18180000000000007E7E000000B0
:1048C80000000000000000000000000000000000E0
:1048D80000000000008080A0C0A000304020C08000
:1048E80080C0A0A0000060A0600000A040A0509878
:1048F800D090882050A850888850A85020608060A8
:1049080000000040E0400000000000800000E000DF
:10491800000000000040002040800040A0A0A0400F
:1049280040C04040E0C02020C0E0E0204020E0201F
:1049380060A0E020E0C02020C06080E0A0E0E0208F
:10494800404040E0A0E0A0E0E0A0E020C00040003F
:10495800400000800080002060E0602000E000E06F
:104968000080C0E0C080E0E0E0E0E000000000007F
:1049780040A0E0A0A0C0A0C0A0C040A080A040C0AF
:10498800A0A0A0C0E080C080E0E080C080806080FF
:10499800A0A060A0A0E0A0A0E0404040E02020202F
:1049A800A040A0A0C0A0A080808080E0A0E0A0A03F
:1049B800A0A0E0E0E0A040A0A0A040C0A0C08080EF
:1049C80040A0A0C060C0A0C0A0A060804020C0E0FF
:1049D80040404040A0A0A0A060A0A0A0A040A0A0EF
:1049E800A0E0A0A0A040A0A0A0A0404040E020409F
:1049F80080E02020A870202070A8202008F030D067
:104A0800100000F0A8A8000000E000000090204876
:104A1800708898984000E0E0E000A0E0E0E04060A6
:104A2800301030606090909090906020602020203E
:104A38002070609010204080F060901020109060EE
:104A480010305090F01010F080E0101090606090DE
:104A580080E0909060F0102020404040609090608E
:104A680090906060909070109060000000000000CE
:104A780000000000000000005060500070705000FE
:104A88000078807008F000F8888888F800C0C8109E
:104A98002040981800C0B098B0C0006020400000C6
:104AA80000000090D8FCD8900000246CFC6C240016
:104AB8000020A870A82000002020F8202000000076
:104AC8000000000080000000F0000000000000006E
:104AD80000606000081020408000708898A8C8888E
:104AE8007020602020202070708808102040F8F87E
:0D4AF80010201008887010305090F8101039
:104B0500F880F008088870304080F0888870F808D0
:104B15001020404040708888708888707088887838
:104B25000810600060600060600000008000008088
:104B350000002040F84020000000F800F8000000C8
:104B45002010F810200070880810200020000000B8
:104B55000000000070888888F88888F08888F088C8
:104B650088F070888080808870E09088888890E0E0
:104B7500F88080F08080F8F88080F08080807088F0
:104B850080B8888878888888F88888887020202068
:104B9500202070381010101090608890A0C0A09050
:104BA50088808080808080F888D8A8A888888888B0
:104BB50088C8A898888870888888888870F08888C8
:104BC500F080808070888888A89068F08888F0A038
:104BD500908870888070088870F820202020202018
:104BE50088888888888870888888888850208888F8
:104BF50088A8A8A850888850205088888888885018
:104C0500202020F80810204080F800CCAC9CACCCCB
:104C15000000CCD4E4D4CC0004781828C800FC40AB
:104C2500A04018202018000000000000F800000037
:104C350000A040A00000006000606000600060000F
:104C450060600000F0A8A8A8A8205020000000007F
:104C55005090B890D0908860505000707050F8888F
:104C6500B898B888F8304C5C6060603C00E0F008AB
:104C75000808F88088482818F804008820208870DB
:104C8500000080C0A090F8003048B4B4483000302F
:104C950048B4B44830FC0098D02058C8008080F053
:0B4CA50088888888F8E8D880D8E8F8F4
:0300000002005E9D
:03000B0002854724
:0C000E00206E06859950D26E32D26F32FF
:0E00230010990AC298206DE385994FD26D3274
:10003800E4F537F534F520F52FC229C22AC268C283
:0800480027C214C215021F0DAE
:03005B00021D374C
:10854700C0D0C0E0C0F0C0A775A700C083C08275C7
:10855700D008758A3D758CEA0532E532700215320E
:108567000530E530640A6026201520E531B40C0B90
:10857700E530B401061288C112A2DBE531B4180B4D
:10858700E530B406061288C112A2DB02873AC2AFF1
:10859700D2C075C07AD2AFF5300531E531641970B4
:1085A70045F531201522C22C7D0A740412AA44EE27
:1085B70024F540142402400E24014008202005DD44
:1085C700E9021D2BD225D22CE5A6600215A678A9B3
:1085D700E660011678B5E660011678B6E660011622
:1085E70078D8E660011620150BE531B40206201A8B
:1085F7000312A4E7302E09E5367005C22E1288480B
:10860700E5366002153678A8E66001160535E535CA
:1086170070021535E590307B0B30E008D278C27BCD
:10862700C200801A307C0B30E108D279C27CC201CB
:10863700800C307D0930E206D27AC27DC202E59015
:1086470044F8F4700B753500302D05C22D1288489B
:10865700E533600515330286DFE590F4540760784B
:10866700F52075330830020E201005201102800610
:10867700E543541FF53320100375A6FF78A8E6706D
:0786870057202D54202E5155
:10868E00301004E536704A20100C201109E535240F
:10869E00F55003753304D21BD2A5D2A675B40C7552
:1086AE00B22278A77655C21C0534202724206821D3
:1086BE0020291E202A1BA21072115015E5206011D0
:1086CE00E5342438400B200026200119D27D753464
:1086DE00C8201558E531702412AA2474E812A9D8BE
:1086EE00802A0287EEE53724FD40E6D27C80DF301B
:1086FE0011DFE53724FD40D9D27B80D275F003849B
:10870E00E5F070DE12933E74E812A9D8E531B40696
:10871E00051294AF8016B40C051294C5800EB412D7
:10872E00051294AF8006B418031294C5E59020E2AA
:10873E000620101020110D78A8E670492010312067
:10874E00113280512027F02068ED2029EA202AE7F7
:10875E00E534243240E1240450DD90877A93D2A68A
:10876E00201002C2A6D2A512883B8045C8A08267FF
:10877E00E5367011E59020E21CE54375F009A495ED
:10878E00355012D22DD2A6201002C2A6D2A5741830
:10879E0012883B801C20340E305A08E54A603C1487
:1087AE00146038128848101B08A25892A5A259923C
:1087BE00A675A700D082D083D0A7D0F0D0E0D0D0BD
:1087CE00202006C5A66003C5A632201003021D2B6D
:0E87DE007581D87438C0E0E4C0E0321288061D
:1087EC0080C6C218B40202D2181293CA3018087488
:1087FC00E412A9D802871A02871578A7E660021638
:10880C002230754079AA7700E579602C14FF760D3B
:10881C0024CE4006EF90888F93F6301C1FEF249CDB
:10882C007410400BEF240A75F0DFA4746F95F0C23E
:10883C001CF5B4C313F5B22278A7767DD21CE4F5EF
:10884C00B4F5B222E57924CE50097628301CED74AB
:10885C001480DC79A1E5799740E2E57979AAC727FC
:10886C002464200E03F4242CFF301C06EFF624366F
:10887C0080BDEF200D02C313F6EF300D022436D26B
:10888C001C80AE78726D68635F5B57534F4B4845E5
:10889C00423F3C39373432302D2B292826242221D3
:1088AC001F1E1D1B1A191817161514131211101050
:1088BC000F0E0E0D0DD2B5C28EAE8DAA8DAF8BAB39
:1088CC008BE4F58DF58BD28E3014012278B6BE0078
:1088DC0007EF24E24002800806E624EC50027614EE
:1088EC00E624F64005E4FEFAFFFB7C007D0A123C10
:1088FC004D7C007D5E123D6D8F7EEE6003757EFFBC
:10890C00EAFC7A33123C61EBF5F0A4E5F0CB8CF089
:10891C00A425E0C5F035E0CB926C25F050060BBBDE
:04892C000002D26C07
:1089300030E7060BBB0002D26CECF5F0A42BFBE594
:10894000F03400FC306C010C78A6E6C39BFF18E6FF
:1089500008F6EB18F618E69CFE18E608F6EC18F692
:10896000301401227A0050040A123EE47C007D6E2D
:10897000123D6D8FF078A2E6A4FBACF0123E83EBC3
:10898000BA0002F404FAE4F8FFEA30E70118E579E6
:1089900060062075031FF4042AF579EF38D275209C
:1089A000E70860037579FF0295D1C2750470F5E59B
:1089B00079F40460EFF57980EE12063DE5BE78A209
:1089C000F624F65007E4F5BEF61239E412063885AF
:1089D000BC2B85BD21E5BEF54824F65008E4F5BE64
:1089E000F5481239E4E5BFF54324F8503B24F34041
:1089F0003712063378A1E5BCF624CD50087432F561
:108A0000BCF61239E4E5BD24F6502824914024E553
:108A1000BF789DF61424FB50087403F6F5BF123995
:108A2000E478B7A6BED25322740AF5BFF5431239D3
:068A3000E480BE75BD0FDD
:058A36001239E480D4B8
:10005E0078FFE4F6D8FDF478D8F6F5A6D220D2B41F
:10006E00D2C075C07A75D75075AE1375AF01758154
:10007E00D875A882D2BC758951D28C7590F875EF5F
:10008E00BC75FDFFC258D2591289B9D2A412A9B7B4
:10009E00C2A4128A3B12AA241292B4C22012A4E75E
:1000AE00121C017F527E0290844F124CC41238EB08
:1000BE0012A88712A9B3745012883B12A9B31288E2
:1000CE004812345312A6A412A88712A9AC753A008E
:1000DE00123478E53A70137F437E06908478124C82
:1000EE00C412A88712A9AC021D2B75A6FFC22B1233
:1000FE0034531289B9121C0112A88712A9AF7520A8
:10010E00001292A9C215121C017F787E0090845FA6
:10011E00124CC47F407E0E78ADE6129EC27E1874DD
:10012E002C129FBF7E1B18E6129EC27E25742C12C7
:10013E009FBF7E2818E6129EC27F497E0E78AEE6DD
:10014E00129EC27E18743B129FBF7E1BE53E129E0E
:10015E00C27E25743B129FBF7E28E53F129EC27F52
:10016E005312979E7F577E0B129D84129E0C7F60BA
:10017E003073417E0BAC5DAB5C129D88129E0C7E83
:10018E0031124D5A7F6A7E1212A22912A8871000D0
:10019E0036100136100236123406D2AC7E3212A759
:1001AE00DAB4E0061234BE02010FDEF2123443124C
:0D01BE00A9AC80F32074097E2BE52E5407B8
:1001CB00129FAC7E17124D5A80BD021D2B021EE0F2
:1001DB008064E53524D2504BE59020E246D0E0D048
:1001EB00E012AA5A803EE53524D25037E59020E242
:1001FB0032D0E0D0E012AA5A306B137F097E009008
:10020B007FB5124CC412A887123B9812514212AA06
:10021B005AE4FFFE9082ED124CC412A88712A9AFCC
:10022B000202D02212AA5AE4FEFF9082ED124CC4B5
:10023B0012A88712A9AFC214C227C268E4F535F51C
:10024B0020753701907FC0120F90900259730200F6
:10025B00FD020A9A0203D80211400202D002030DDA
:10026B0002026EE4F535F520753707908007120F03
:10027B00909002807302024102034A02037702024A
:10028B00AC02026E02026E02372302391C02029E7E
:10029B000203A41238B81239D512A4E780C512395B
:1002AB00E4E4F535F520753702908051120F9090EC
:1002BB0002BE7302026E0206680206CE0207250218
:1002CB00076A0207AFE4F535F5207537059080878F
:1002DB00120F909002E273020241024F08024F4D3F
:1002EB000250E00202D002030602501F02508502A8
:1002FB000A630202D0020A490204707F2E12098F90
:10030B0080C3E4F535F5207537069080EE120F901B
:10031B0090031F73020241020AA0020AFA020B6B3E
:10032B00020C38020C6A020CE102030D02034002BC
:0C033B000D14020DB97F4912098F80C615
:100347001239E4E4F535F520753703908151120F22
:100357009090035C7302026E020838020491020453
:100367009C02089B0209F70205180204AB1239E444
:10037700E4F535F520753704908193120F909003BB
:10038700897302026E0204B60204C10204CC020998
:10039700AC0204D70207BE0207C20204E6E4F53541
:1003A700F520F5379081D6120F909003B5730202AE
:1003B7006E0203C40203C90203CE0203D3123AF743
:1003C70080DB123A6980D61239EF80D11237298043
:1003D700CCD25712AA5A1210371203E60202417FF3
:1003E700177E0290045A124CC47F377E0290046530
:1003F700124CC4AC5DAB5C7F427E04129E041206B5
:100407004C85BC6285BD63E5602562FBE5613563AC
:10041700FC7F227E04129E0412A887100008100198
:100427001010022080E11562E562B4FF0C156380AD
:10043700080562E56270020563E53524F550C87565
:10044700330180C312064C128A6A8562BC8563BD7C
:100457000239E4534554204845494748540047501A
:100467005320484549474854001210A912A887103D
:10047700001510010280F87F637E05907FB5124C4E
:10048700C412A887123B740202D07F13A20D120474
:10049700F1920D80097F1CA20E1204F1920E120533
:1004A7000C02034A7F3FA25E1204F1925E80EF7F47
:1004B7000AA2081204F19208801F7F13A20B1204EC
:0904C700F1920B80147F1CA209C4
:1004D0001204F1920980097F2EA20C1204F1920CF1
:1004E00012050C0203777F49A20F1204F1920F80CC
:1004F000EF8F1F921712066012063885BC2B85BD40
:1005000021AF1F1F7E39125978A217221206388593
:100510002BBC8521BD0239E420371412063385BE79
:10052000121205451206338512BE1239E480057F8A
:100530003612053702034A7E03908227124CC412FA
:10054000A88702A9AF75A6FF12AA5AC22F74071274
:10055000AA468FF0740612AA46102FEFEF2512C399
:1005600095F0FD78D8E6C4540F2DA2E7923D4010D7
:10057000FD24CD50027D32AC05C3743F9DFD800F3C
:10058000F404FD24C850027D37AC0574402DFD7F76
:10059000401297967E1212A94C0EBE1EF91F303DD6
:1005A000020F0FEF6D70EDE536700A753606EC251B
:1005B00013F5148C131205CE12A887100007100132
:1005C00008300207221512800205120205457F3706
:1005D0007E28742E129FBF7F347E21740A303D0125
:1005E00004129FDCE514FC249C50027C63EC75F043
:1005F0000A84C0F07F347E2D129FDCD0E07F377EEE
:1006000036129FAC7F437E1E129D847E00E512123F
:020610009F1B2E
:100612007F057E029081FB124CC47F6D7E01908229
:1006220006124CF57F747E04908218124CF502106B
:100632003775C6F8802175C6F9801C75C6FA801711
:1006420075C6FB801275C6FC800D75C6FE800875E6
:10065200C6FF800375C6FD75C70375B90122743FD5
:10066200129F8D02A8877F0A1206607E2A12347BAF
:1006720012063DA8BF12069D1000121001051002BD
:100682001580F508E824E750EC781880E818E8307F
:10069200E7E3780080DF88BF0202A97F097E059028
:1006A200807BB80C03908081124CC47E27E53D28E4
:1006B200240C75F01884E5F0129E577E33743B12B9
:1006C2009FBF7E35E53E129E5702A8877F13120612
:1006D2006012063885BC2B120702100008100105B3
:1006E20010021780F2105C07205D0BD25C80E810CC
:1006F2005DE5D25D80E1D25C80DD852BBC0202A982
:10070200205C10205D189082337F127E23124CC42D
:1007120002A887908247205DF090823A80EB908217
:100722004080E67F1C120660120638A8BF12075DE1
:1007320010000810011110021A80F2E824F7500389
:100742001880EA780880E6E824EC40030880DE7826
:100752001480DAE8F5BFF5430202A97F1B7E2EE87A
:100762002323129E5D02A8877F2512066012064788
:02077200A8BC21
:10077400E81207A612A88710000810010D10021F26
:1007840080EEE824E050E9188006E824CF40E10830
:1007940012064788BC1239E4D21512A4E780D102AC
:1007A40002AC7F247E3724E2029EC87F2EA20A1266
:1007B40004F1920A12050C0202ACD23D8002C23D41
:1007C4007F40303D027F3712066012063DA8BD30DF
:1007D4003D02A8BC12080210000810010D100212FC
:1007E40080F218B8FFEE787D80EA08B87EE67800DB
:1007F40080E2203D0488BD800288BC0203747F3FF0
:10080400303D027F36E823129B3D75F06484C0F0CE
:100814007E20129FAC7E26742C129FBFD0E07E29CE
:10082400129E577E3590824D305D03908250124C5B
:10083400C402A8877F0A120660120633A8BCE81215
:10084400086D12A88710001010010510021280EE26
:1008540018B8FFEA783280E608B833E2780080DE20
:10086400E8F5BC79A1F7020347305C01237F097ED8
:100874002375F00A84C0F0129EC87E2D742C129F3A
:10088400BFD0E07E2F129FA50F7E35908253305C3F
:1008940003908442024CF57F2512066012063DE562
:1008A400BE7F247E2C1259CDF5BE79A2F7020347F0
:1008B400120638E5BE7F097E3A029FAC12063DA8B7
:0A08C400BF12069D12063885BC2BFA
:1008CE0085BD21120702A8BF12075D120647E5BCBF
:1008DE001207A67F2DA20A807512063885BC2B85BD
:1008EE00BD217F12A20D12095C7F1BA20E12095CA4
:1008FE00120633E5BC12086DA8BF120A3512063D6A
:10090E00E5BE7F247E2C029FAC7F3FA25E803F120D
:10091E00063DA8BCD23D120802A8BDC23D12080277
:10092E00120633E5BD1209DF12063885BD217F0997
:10093E00A20812095C7F12A20B12095C7F1BA2098E
:10094E0012095C7F2DA20C12095C7F48A20F744E17
:10095E00400274597E3A029FBF1253327F6E124F7D
:10096E00CB7F2D800E120638E5BE7F097E3A129F90
:10097E00AC7F487E1E90825730530390825C024CAF
:10098E00C41206601F12098112A8871000081001F8
:10099E000510020980EF1053ECD25380E8227F2518
:1009AE001206607E35120633A8BDE81209DF12A8C2
:1009BE008710000810010D10021280EE18B809EA17
:1009CE00787880E608B879E2780A80DE88BD02037E
:1009DE00747F247E2975F00284C0F0129E5DD0E0F3
:1009EE0075F005A47E3B029FAC7F2E1206601206A8
:1009FE0033A8BFE824FA40033037027803120A35D1
:100A0E0012A88710000810010D10021280E518B808
:100A1E0000E1780580DD08B806D9780180D5799D8A
:020A2E00E8F7E7
:100A3000F5BF0203477F2D7E2C7420B80502742E6B
:100A4000129FBF7E32E8029FACD26875480A12340A
:100A50007BD214121D631254501225F5C26B120181
:100A6000F180F3D2147515011252EC75B901E5BC91
:100A700004601C12540075A6FF12545C121066121A
:100A8000A887124DD010000F5005124EF880E705D0
:100A900015E515242050D10202D0120AA602024107
:100AA000120AA602030D120AB21206388548BE02C7
:100AB00039E4121D55121D6F1244C412AA5A9082B5
:100AC000771267431266FB12105B12A887100008AA
:100AD00010011110021B80F50548E548640A7002F8
:100AE000F54880D11548E54864FF700375480980D2
:100AF000C4854849121D6FE55822121D5585484985
:100B0000C250E558B40F02D2501244C48038D227E4
:100B100075480A121D631244C412AA5A12668490C0
:100B2000828120290390828C1210D4C26A1225F58A
:100B3000106A0280E1C2271252C4854948120EBFD2
:100B4000121D6F1244C412AA5A12674020500E128E
:100B500010B412A8871000101001B380F8121066AC
:100B600012A88710000280FB02030D121D55E558E4
:100B700030E7137F1B9082617E05124CC412A88758
:100B800012A9AF02030D121D6F1244C485594912F8
:100B9000AA5A12104B90828C12674312670512A852
:100BA0008710000810010A10020C80F5120C038057
:0C0BB000DB120C1080D612AA5A12104B57
:100BBC0090829712674312670512670912A8871073
:100BCC00000810010A10020C80F5120C1C80DB12BC
:100BDC000C2A80D6120E85121D6F1244C412AA5A0A
:100BEC00907ED412674312108E12A8871000051045
:100BFC00028880F802030D0559C3E5589559500336
:100C0C00755900221559E55964FF7003855859220E
:100C1C000549D3E5491495584003754900221549F7
:100C2C00E54964FF7005855849054922121D55E5B3
:100C3C005830E7057F24020B75121D6F1244C41245
:100C4C00AA5A9082A21267431210BF12A8871000F2
:100C5C000A10010280F8120F2E80DE02030D121D05
:100C6C0055E55830E7057F2D020B75C26B7559FFA2
:100C7C001244C412AA5A121037E55930E703121065
:100C8C005B9082AD12674312671512A887E5582056
:100C9C00E70610000810011110021B80F00559C363
:100CAC00955950CF7559FF80CA1559E55964FE7096
:100CBC00C285585980BDE55920E711D26B75A70044
:100CCC00758307C4F582E0B2E7F080A7306B03129E
:100CDC000EDC02030D121D55E55830E7057F360278
:100CEC000B75121D6F1244C412AA5A9082B8126767
:100CFC00431210A912A88710000B10010280F812E1
:100D0C000F23120F5802030D121D55E55820E7084A
:100D1C007F5190826C020B7812AA5A9082CD126786
:0A0D2C004312106612A8871233EE7E
:100D3600D2AC10001FE55830E7F8306DF5120E34CE
:100D46007E207F0050139082E3124CF512A8871282
:100D5600A9AF80CAC2AC02030D1B8B13907FB512DC
:100D66004CF512A887C26B7B007514B8120F1812C7
:100D760053CF1253815025A814E824384004A60105
:100D860005140BC3E5139B50E678B8120F5A306B67
:100D960003125142121D6F1244C48082125332E56F
:100DA6001660E6D26B12542CC003125303D003A96B
:100DB6001580C4121D55E55830E7057F5A020B759C
:100DC600121D6F1244C412AA5A9082C212674312AD
:100DD600108312A88710001B10010280F8120DFC68
:100DE6009082D850039082E312674312A88712A913
:100DF600AF80CD02030D1233EE12A7A1745212A7D3
:100E06004B745412A75DE5580475590012A7901249
:100E16004D8540161252C4125400124DD0400B0597
:100E260059C3E558955950ECC322C2ACD3221233AC
:100E3600EED2AC12A7D5C5F060F0C5F0B440F412FE
:100E4600A7DAB4400312A7DAB452DFF53812A7DAEC
:100E5600B454D712A7DAFA60D124EF40CD12A7DA3C
:100E6600E53870C612A7DA12A7DA124D6C7B0012AB
:100E76004E5840B61253DF0B124D6CDAF2C32212F3
:100E86000F69E55924C8F88602E54924C8F998602F
:010E96001348
:100E9700146010500F18E608F618E86970F7A702F3
:100EA700120F5822E559640F60F91908E618F60879
:100EB700E86970F7A70280E8120F6978C8C250E6A0
:100EC700B4FF02800708B8D8F6D25022B8D702D2AA
:100ED70050A615807C78B8120F6BE4F9F5A77583D7
:100EE70007E9C4F582E030E70AE924B8F824384076
:100EF7000276FF09C3E5589950E7120F2378B879AE
:100F0700C8E6B4FF028002F70908E8243850F280E7
:100F17004079B877FF09E9243850F82279C877FF74
:100F270009E9242850F822120F69C23D78D7B6FF85
:100F370004A900D23D18B8C7F5203D0279D8197821
:100F4700C8B6FF0122C3E8995007C6C7C60819806B
:100F5700F478C8120F7A12543E12543E12543E02CD
:100F6700543E78C8120F7A12541A12541A12541A8D
:100F770002541A75C703E54875F004A42480F5C622
:100F87002212AA5A124CB0800612AA5A124CB4E581
:100F970037603014602A14602214601A1460121427
:100FA700600A146002801C12097380171209678097
:100FB7001212091D800D1208E780081208C080036D
:100FC7001208B412A88712A9B3121037D234E4F565
:100FD700B4F5B2A81F08E814C23BB51D02D23B7591
:100FE700F007203C0375F009A4FF203C010F7E00A9
:100FF7007420303B02743E129F8DD8DA12A887E521
:101007001D10000810010D10021080C0651F60BC84
:10101700051D80B860B6151D80B275F003A42212B5
:101027004FF87E05745B129F897E1D745C029F8951
:101037001210267E34901042024CF553454C001294
:101047004FF880031210267E31901056024CF54E51
:10105700455854001210267E319082EE024CF5124C
:101067004FF87E008005124FF87E2D9082EE024CDD
:10107700F51210837E319082FA024CF51210667ECB
:101087001A9082FF024CF512106680BB1210667E22
:1010970018908304024CF51210667E1A90830A0298
:1010A7004CF51210667E1A90830F024CF5121066EB
:1010B7007E1A908315024CF51210667E1890831BDA
:1010C700024CF57F7B7E00908321024CF57F007EEA
:1010D70020124CF502A887128CB6120656E5BDF50C
:1010E7005EF56CE5BCF55FF56B756A007561FF75BC
:1010F700A704900700128C62B4FC12E582C313F5B3
:1011070061E56CF0E56BF0E58260168005B4FF02DF
:10111700800F128BCAE56C655E70DAE56B655F70F0
:10112700D475A70022E560758307C333F582E0A372
:10113700F56CE0F56B756A0022D214C21F1210DE3F
:10114700756000E561B4FF1612AA5A90833D7F0AC5
:101157007E05124CF512A88712A9AC020241C210F3
:10116700C21112AA5A121037301F0C7F077E009047
:1011770082F3124CF580647F007E01C3E560129F05
:101187002B7E0E7428129F898560487407F51FFF10
:101197007E00743E129F8DE54812112E1295ED12B6
:1011A70016B60548C3E5619548FD401CE51F2407B1
:1011B700F51F24C850E17F387E01ED04129F2B7E76
:1011C7000E7429129F89800DE51F2407FF7E019069
:1011D70082ED124CF5201F031216F912A887100092
:1011E7001910012C10020280F51201DD301F3D029B
:1011F700022F101F02D21F021165E56160F4E5603E
:1012070065617005201FF080E9201FE6056080E713
:10121700E56160DEE56065617005201FD580092006
:101227001FD5E560700280CA156080CB1210DE12F0
:10123700112C1295ED1217EB756A10128C491218C2
:10124700A290834B124CB0120FD09012557302111B
:101257006502245002127E0212611210A912A88799
:0E1267001000C910010280F812112C128C62C6
:10127500C2E2FF128B05021140C25312112C1295C6
:10128500ED753700908364120F90901293730212DC
:101295003302148002148502127E0212BA0212BFB2
:1012A50002127E0212FD02130102130502130C0243
:1012B5001310021314123420800312340D780A120D
:1012C50013DD740412A75B12141C12A7891214579C
:1012D500128C49128C75128B82128D8C12156DD55C
:1012E500150C75150A12146A12168012A7891002B8
:1012F50004E57F70DB021233780A800678048002E9
:101305007801123420800D780A80067804800278EE
:101315000112340D1213DD740412A75012141CE5CA
:101325004812A737742A12A75D12A75D12A75D128E
:10133500A789121457128C49128C75128B82128D43
:101345008C12156DD5154885481512146AE51C12C1
:10135500A737E51B12A737E51B2548F51BE4351C08
:10136500F51CE4A27792E7A27492E0A27392E112CF
:10137500A737AD75AC74AB73E57DC412139EAD781C
:10138500AC77AB76E57D12139E12169E12A78910D7
:101395000204E57F709F021233540F2375F0058414
:1013A500F8C3EB33FBEC33FCED33FDC3EB33FBEC64
:0F13B50033FCED33FD20E713EB28FBE43CFCE4B5
:1013C4003D12A737EC12A737EB02A737C3EB98FB04
:1013D400EC9400FCED940080E8884812106DE4F56C
:1013E4004AF549756A20751501128C49128B82D50C
:1013F400150E854815E5492401F549E4354AF54AB1
:10140400E57F70E5744012A74B747812A75D74638E
:1014140012A75D741602A75012165BE56012A73777
:1014240012112C1295EDE53A12A750E53B12A75084
:10143400E53C12A750E53D12A750E53E12A750E542
:101444003F12A750740112A737E54A12A737E5499E
:1014540002A73712112C756A20E4F51CF51BF5144C
:10146400F51375150122753800E51412A737E51335
:1014740012A7370513E513700205142212342080D5
:10148400031233F112106D1215B612A9B7756A2042
:1014940075150175A6FF754A01128BEF128B821226
:1014A4008D8C12156DD5150975151E12159112A97D
:1014B400BD121680E57912A737E57EC33350027456
:1014C400FF12A737E57112155212A737E57012A75C
:1014D40037E57B24ACFFE55F340912A73DEF12A783
:1014E40037E51520E033857D56E412A737E52EC491
:1014F40012A73D12A79812A9BD10021A3055947470
:101504004012A75D744512A75D744F12A75D74461F
:0F15140012A75D12A798021233E55612152CC4C8
:10152300FAE57D12152C2A80C2FBC4121539232338
:10153300CB1215392B22540FFC24F650027C009059
:101543001548EC932200000101010202030303FA90
:101553002440400A24804003EA3322D2E72274FF66
:101563002220E703C3132224C022E53F701F7F7BA1
:101573007E0078AEE6129F15EE2404FE743A129FA5
:101583008DEE2404FEE53E129F0F12A8872278AE4B
:10159300E612A750E53E12A750E53F12A750E4120A
:1015A300A737E412A737740A12A73774C012A737F4
:1015B30002A798744012A75D745412A74B744E127D
:1015C300A75DE412A73712165B741612A750E53D08
:1015D30012A750E56012A73712112C1295ED78ABC4
:1015E300E60812A750E60812A750E60812A750E62D
:1015F30012A750E53E12A750121BE8E51212A7509E
:10160300E51112A750740112A7379083DE1216A8B2
:10161300756A10128C49057F057F787F12A7307891
:101623007B12A730787D12A730787712A730E4FEBB
:10163300FF780712A73012A730E57412A737E575B4
:1016430012A737E412A737E573C333500274FF12AE
:0E165300A73712A73002A79875C70375C6FF08
:1016610075B901C217751D0085BC1C85BD1B85BEE2
:101671001A85BF19123BE7EE12A737EF02A737E52C
:101681007512A737E57412A737E57312A737E57806
:1016910012A737E57712A737E57612A737E55E126D
:1016A100A737E57A02A73775A700E493700122A353
:1016B10012A75D80F5AF1F7E0478ADE6129F0F7E05
:1016C1000C742C129F8D7E0E18E6129F0F7E1A78D5
:1016D100AEE6129F0F7E22743B129F8D7E24E53E63
:1016E100129F0F7E2FE540129F157E37743B129F8C
:1016F1008D0E0EE541029F0F75320012112C1295CD
:10170100ED857946787A79641296067464123FC23F
:101711001217EB756A20D23D128C49128C75121882
:1017210022303D09307406C23D8E1E8F1FE57F6059
:101731002BE54C24FFF54CE54D34FFF54D454C6050
:1017410005128BA080D2751D3C128C49128C75122A
:101751008B82121822E57F6003D51DED121883904C
:10176100189B129FED203D0DAE1EAF1F12188390E6
:101771001894129FEDE546FD700B908519305D11AF
:10178100908515800C047010908515305D0390854F
:10179100117F38122FF8804BE4FFFC7E05305D0489
:1017A1007E027FB3123D6DAC06AB07123C377F382A
:0D17B100C23DE51C6007D23D7E2C129F7AE0
:1017BE00E51B203D026007D23D7E30129F7AE51A6E
:1017CE00203D026007D23D7E34129F7AE5197E38A5
:1017DE00129F7A122FFDE53224C850FA22E5407589
:1017EE00F03CA42541FFF54CE435F0FEF54D7C00B0
:1017FE007D10123D7A0F8F4BAF4CAE4D7C007D3C71
:10180E00123C4D7C00AD4B123D7AEE4F70010F8FA6
:10181E004C8E4D2278647973C2D1121839FF7867D5
:10182E007976D2D1121839FE02A94CC3E796FB087D
:10183E0009E796FC0809E796FDA2E79217500312F6
:10184E003EFC75135A30D10E751320B217AA4712EB
:10185E003C81AB04AC05E546600B04600BAA461256
:10186E003C98EB03FBEB03FBEB543FFBE5132B2008
:10187E0017029B9B22EE141430E701E4FEEF1414C2
:10188E0030E701E4FF2205057088A8887005052061
:10189E0020F8202075320012AA5A7E1E7F1C12A933
:1018AE004CDFFB12A94C7E1E7F1C12A94CDEFB7E68
:1018BE001D7F1D12A94CDEFB7F007E2178ADE61246
:1018CE009F0F7E29742E129F8D7E2D18E6129F0F6C
:0418DE007E35742EB1
:1018E200129F8D7E3918E6129F0F7F077E21745456
:1018F200129F8D7E25744F129F8D7E2D78AEE6123B
:101902009F0F7E35743A129F8D7E39E53E129F0FEE
:1019120078AE121BE87F0E7E21744C129F8D7E25BD
:101922007441129F8D7E2DE512129F0F7E35743AFF
:10193200129F8D7E39E511129F0F7F157E2574440B
:10194200129F8D7E2DE540129F157E35743A129FAF
:101952008D7E39E541129F0F7F1C7E2F85715412B7
:101962009C087F217E01908435124CF57E0EAC7767
:10197200AB76129DC17E2B85795F85787B12A28220
:101982007F287E01908439124CF5751D2B751E102F
:10199200E574121B9C7E25742F129F8D751D2D756B
:1019A2001E2BE575121B9C7F2F7E0290842D124CFC
:1019B200F5E5736003121A477F367E029084251282
:1019C2004CF5E572121A47121ADF12112C756A20B1
:1019D2009004E6E56CF09004E7E56BF0AE4DAF4C99
:1019E2007C007D40123D7ABF00010F0FAC07AD07AE
:1019F200E4FED23D128C49128C75121A88E57F6082
:101A02002CE54C24FFF54CE54D34FFF54D454C607B
:101A120005128BA080DE751D3C0E128C49128C754E
:101A2200121A8DE57F6006128B82D51DED121A5DAA
:0E1A32007F781297A87F767E007430129F8D09
:101A4000E53224C850FA227E21129B3D129F2B7E44
:101A50002F90843D305D03908442024CF59004E663
:101A6000E0FD9004E7E0FCC3E56A9420FBE56B9C95
:101A7000FCE56C9DFD50032410FD123E6C9004E8C3
:101A8000EEF09004E9EFF022DD03AD040E7F78E57F
:101A90005E20E72AE57A8549F0A4A9F0E57A854A2F
:101AA000F0A429F9E435F0FAE55E8549F0A429E4CB
:101AB00035F02AFAE55E854AF0A42ACF9FFF12A9E5
:101AC0004C103D18C3EF9B50131BEF6B600E8F0142
:101AD0008B0712A94C1FEF6970F8AF01AB0722907A
:101AE00083EA305C03908403754A40754900AF7601
:101AF000E577FE20E76B7005EF24105064EF24A813
:101B0000EE34FD40119083EF305C03908407754AFA
:101B10001975499A8075EF2450EE34FB401190837B
:101B2000F4305C0390840C754A0C7549CD805CEFF1
:101B300024A0EE34F640119083F7305C03908411BA
:101B4000754A067549668043EF24F0EE34F1401380
:101B50009083FA305C03908416754A04754944807A
:031B60002A8028B0
:101B6300EF2490EE34E840119083FD305C039084C1
:101B73001B754A0275498F800F908400305C039077
:101B83008420754A0175499A7F407E00124CF57F87
:101B9300461297A87F5F0297A8AE1E75F064305C6B
:101BA3000375F03284C0F0F87004EE2404FEE51DE2
:101BB300129F8DEE2404FEE86007129F7AEE240440
:101BC300FED0E075F00A305C0375F00584A8F012CE
:101BD3009F7AEE2404FE742C129F8D0E0EE8305C67
:101BE3000123029F7AE53E2541F51124C45003F5F4
:101BF30011D3E63540F51224E85002F51222D2340F
:101C0300128848C21012AA5A7F057E099084461290
:101C13004CC47F147E08901C3D129FED7F2B7E01E8
:101C2300901CA5129FED2037107F277E29E53F20CA
:101C3300E0010E901D17129FED22113007FE1FE0E9
:101C430001E101F80F00061B00F80C00180E007CE0
:101C530010007006003C2000E006003E4001E00456
:101C6300001E8003C004001F0003C004000F000710
:101C73008000000F800780000017800F00000027FE
:101C8300C00F00000043C00F00100083E00F0020CE
:101C93000301F00700C00F01F80383007F87FE01F3
:101CA300FC000E3E180000030000000018000003B3
:101CB30000000000380000000000000030000000B9
:101CC30000000000FC761F0E1C6030ECFCBC3F17CC
:101CD3002DF0F978613866264F619A706070C60EF0
:101CE3001EE330E06060C60C1CC360C0E0618C0C76
:101CF30018C7C0C0C0E18C1C39C611C0C4C19C99AF
:101D030031963180C8C1FF1E31E7E180F0C0EE1C7F
:101D130031C38180061630918828928849249049DE
:101D230027909248A0E3C8BCC2AF74FE12883B7FE1
:101D33006412A9BFC2B480FC75C703E54875F004FB
:101D4300A42480F5C6C23C75B901E5BC047002D277
:101D53003C22120638E5BEF54824F65003754800C8
:101D6300753400753703C228D229D22A75C703E513
:101D73004824E75003754800E54875F004A424801F
:101D8300F5C6751607751700C23C121DB0121DB0BB
:061D9300121DB0121DB08C
:101D99008517581558755900E548B40A09E558607A
:101DA90005F46002055922203C1D75B90105C6AA32
:101DB900BCABBDACBEADBFEA121DD1EB121DD1EC5F
:101DC900121DD1ED121DD122203C07F515B4FF03D8
:101DD900D23C22C0C7C0C61252EC75A7048516832F
:101DE900E517C4F8F58275B90105C6E5BCF0C582E9
:101DF900F82406F92403C582E5BDF0E5BEF0E5BF88
:101E0900F075B90105C6E5BCF0E5BDF0E5BFF085A3
:101E190016838982E4F075B90105C685BC1385BDB1
:101E290014E4F0F08882E5BEF0E5BFF075B901E58C
:101E3900BCF0E5BDF0E5BEF0E5BFF0758306E5173A
:101E490023541E24B0F582E513F0E514F075A700BC
:101E5900D0C6D0C70517221289B978BEA64808E4AA
:101E6900F6F55908761808F6C23608760A08F6060D
:101E79000876BEC225C254C255128CCB121D63C24C
:101E890029C22AC227C268E4F537F52EF534F52FA1
:101E990078A8F678AAF678B6F678B5F6789EF67840
:031EA900B8A65E7A
:101EAC0008A67AC233C238C240C223C222D241C26F
:101EBC0042754601C23AD221C219C226C23485707B
:101ECC005778BA7401F608F608F608F6E4F542F508
:101EDC0041F54022121E6012655C75440312347881
:101EEC0012779AD54403021D2B201EF1789F768021
:101EFC00754A00128A78D210753950C211C213C2B9
:101F0C0012123406C24675A60A1292A920120312A6
:101F1C0023ABE5A624FA400612344375A60A202505
:101F2C0011E54375F00AA4242295355007E590205D
:101F3C00E202806B201E1DE532241040172046144F
:101F4C002428500D30410AE537B40205126C0BD22F
:101F5C00461225F5D2AC306DB912A7E4B4E0B31239
:101F6C0034BE304108E537B40203126C0B12207CEE
:101F7C001225F5126F97128E301225F512655C3012
:101F8C00121A128B1FE5510404F57F24FE400375D1
:101F9C007F02C277E54024F05002D255021F0D7526
:101FAC00A6FFC210301203121FBEC212752F000200
:101FBC0000FD12349C128CA212AA5AE47E057F1EDC
:101FCC00908482124CC412A88712A9AFD214D220CA
:101FDC00120638852BBC8521BD75B90575B9021261
:101FEC008CACD255128BC47F00128B05D220128C74
:101FFC00ACE56A6005128B8280F7857A62D220127A
:05200C00065685BEBC74
:1020110085BFBD856BBE856CBF75B90575B9028578
:10202100BD6C85BC6B756A20128CA2122221128CA8
:10203100AC756A00128C49E57064FE70397570FCEC
:10204100854077854178851F797818797A129606C7
:10205100128B67D22012A9BD128CAC756A10128C3A
:10206100498554717F087810797212960885627CCF
:10207100855E7D128B67C220C21422300A012212B2
:1020810034201221CD745212A75D744D12A75D74D4
:102091004312A75D1221DC12A7AA744120740274B5
:1020A1005612A75D12212912217312A7AAE53C122B
:1020B100A750E53B12A750E53A12A7501221A912E9
:1020C100A7AA744512A75D1222121221CD744712DC
:1020D100A75D744712A75D744112A75D1221DC123E
:1020E100212912A7AAE43074010412A75B12A7AA3E
:1020F1009004C3E012A75012A7AA9004E4E075F07F
:102101000A84AFF012A75012A7AEEF12A75BAC5E24
:10211100AB7A1221EEAC5DAB5C1221EE12A7AA12D2
:10212100A7AA1222120234067875C23D1221347810
:1021310078D23D12A7AA12577C303D05E51E12A7A1
:102141005BE51D12A75B1221B6E51812A75BE57DC1
:10215100203D01C4540F12A75B12A7AA303D097498
:102161004530170274578007744E301702745302BA
:10217100A75D2074081221A91221A9802775A7043F
:0C2181009004BFE0FCE0FB7A1B123C6FF6
:10218D007832123E11123C371221B39004C1E0FC9B
:10219D00E0FB123C371221B375A7002212A7AAE467
:1021AD00F51AF519800D12A7AAE51C12A75BE51B00
:1021BD0012A75BE51A12A75B12A7AEE51902A75B82
:1021CD00742412A75D744712A74B745002A75D12B9
:1021DD00A7AAE53D12A750E53E12A750E53F02A77D
:1021ED00501257D812A7AAE51D12A75D781CE6124A
:1021FD00A75B18B817F812A7AEE412A75B12A7AA2F
:10220D00744D02A75DC038742A12A75DD03812A78D
:10221D008902A9BD78107F0EE4F608DFFCF564F5A0
:10222D0065F567F5687515FC751AC0751DC0756681
:10223D0040756940754A01128BEF3055030222DD5E
:10224D00128B82E571B510004002F510E57EB511D7
:10225D00004002F511E512207502E513C395795082
:10226D0006207545857913D3E57A9514E5156480B7
:10227D00FFE55E64809F400C857A14855E15857B35
:10228D0016855F173074ADC2D1786479731222BB95
:10229D00786779761222BBD2D1781879731222BB66
:1022AD00781B79761222BB808B85791280B9D3E7A2
:1022BD00960809E7960809E66480FFE764809F2089
:0722CD00D101B3400AE7F65E
:1022D4001819E7F61819E7F622E51AB4C00E787350
:1022E40079181296067873796412960678187964C8
:1022F400C2D112234C7418123FC2AE1EAF1F781BFA
:102304007967D2D112234CC3E51F9FE51E9E50046A
:102314008E1E8F1F7EFF7FFFAC1EAD1F123D7A7A8B
:1023240004EF8AF0A4E5F0CE8AF0A42EFEE435F0A2
:10233400BEFF011E60051460057EFF8E1F22EE7E27
:102344000020E7F77EFE80F3C3E697FB0809E697D3
:10235400FC0809E697FD1818191930E703123EFC2A
:10236400C3EB33FBEC33FCED33FDEB33EC33FBED30
:1023740033FC30D105AA47123C980BBB00010C7505
:102384001E03751FFFEC24FC40048C1E8B1FE627E4
:10239400FB0809E637FC0809E637A2E713F618EC50
:1023A40013F618EB13F62210131978B5E624FA4045
:0723B40012E57124F6400858
:1023BB00E57924F64002802606068022D220753667
:1023CB0012D22EE4F534F537F55A128CFD1223EFA9
:1023DB00C219D236C257126F34126F61D212121E4B
:1023EB00CAC22022D214122445E6F008DFFB857AFC
:1023FB006212243B7570FE783A7971129606128B35
:10240B006712243B85627A855E7B75C70375C6FEB2
:10241B0075B90185BC7E85BD7F7570C0128B671247
:10242B002445E0F608DFFB75A700757F01C2142277
:10243B0074FF7870F608B880FB2275A7049004F03F
:10244B0078707F102212112C1295ED128E169004BB
:10245B00EAECF09004EBEBF01233F1751F0312155D
:10246B00B67F6412A9BFD51FF5121E6012AA5A12AD
:10247B00A887C25AC258C259756A20128BEF123FF5
:10248B00C0754A01753901C210D211D214D236D29D
:10249B0012128CFD126F34126F6175A6FF7536091F
:1024AB00753200E54375F00BA4241995355020E5E2
:1024BB009020E21BC211C21212AA5A12A887E4F58D
:1024CB0035F52FC22D7E0612A9B9C202021233E5D1
:1024DB004A20E016128DFC1233F112A7A174491297
:1024EB00A74B780412A73012A789C221B40202D2DB
:1024FB0021128BEF126F9730261112452612655F52
:10250B00753606E53670FCC226808F12655C122587
:01251B00F5CA
:10251C00E54A20E021B40209753900E53670F980EE
:10252C00E7E53960E3FD24E240020539128BEF2028
:10253C0026C7DDF880D27539001233F1D2ACE536FE
:10254C00602712A7DAB440F612A7DAB4400312A738
:10255C00DAB44915F53812A80FFC12A80FFBAD38E8
:10256C0012A80F6D7003122579C2AC809BC3900426
:10257C00E9E0FF9B9004E8E0FE9C50048E048F037E
:10258C008C148B137A10123C6F74202BF56A900408
:10259C00E7E03CF56B9004E6E03D540FF56C754AB2
:1025AC0001128BEFAE14AF137C0E7D10123D7A8F9F
:1025BC0040AE04AF057C007D3C123D7A8F418D42CC
:1025CC009004EBE02513FF9004EAE03514FE7C0E3A
:1025DC007D10123D7A78AEA607AE04AF057C007D67
:1025EC003C123D7A8F3E8D3F2210002910010D10B8
:1025FC00020D20783020790A207A172202274F0208
:10260C0026AFE53760061460060227BE0227630278
:10261C0027950226D3E53724FD500A24FD400302FA
:10262C0028310227FF201145753400201203D213E4
:10263C002278A9E6700E760AD277D226753614D295
:10264C002E028CF2200B25204122E537B4021DE628
:09265C00B4050B126F34126F611A
:1026650075360A8009B4080B126F3475360578A9DA
:1026750016D22E2210780122753900E5342438400F
:1026850007754A0175340022700AE54A30E0F27593
:102695004A0280F0146008754A06126F618006755B
:1026A5004A04126F3475390180DA302909C229D2FA
:1026B5002A7559008005302A0CD2291266F1126656
:1026C500BF7534002220687C302703D26A22D222CB
:1026D5001229B4107A0122E53424384009753700EF
:1026E500C24275340022700BC242E4C53770F3054F
:1026F5003780EF04F53724FA5009C242753706D200
:102705002880DFE5376402602DC242C228E5372400
:10271500FD2324BEF879C4E7F9A74809A75979C468
:10272500E8F78648088607E537B4040375481812A4
:102735001D6F8F5980AC204204D24280A51041A262
:10274500D241809E122990022938E5376010146025
:102755003F14606524FC400302289C022872D223A2
:10276500122F7810790122E5342438400775460187
:1027750075340022700EE54624FE40F1E54660ED15
:10278500154680EC04F54624FA50E575460580E0CB
:0E27950010790122E53424384008D25BD208C6
:1027A3007534002270083008F3105BF480EE147067
:1027B30004C25B8002D25BC20880E510790122204B
:1027C300412CE5342438400AC258C259C25A7534E0
:1027D3000022700B205AF1D25AD258C25980EFD23C
:1027E3005AC258D25914700280E4D25880E078B8A3
:1027F300A65E08A67A753605D22E80D230122B1229
:10280300672B055BE55B75F00B84E5F0F55BE55A3B
:1028130024F64009E55A955B5003755B0012672F58
:1028230012A887E5346003D534D275340022C24040
:102833003029030228DC1266ED126701102A2405F1
:1028430059C3E55895595005755900801BE558B48F
:10285300FF0375590012671512A887E5346003D585
:1028630034CC2275590080EDD22A1266F180E9300A
:10287300122312672B155BE55B30E70C755B0AE5EA
:102883005A24F64003855A5B12672F12A887E53452
:102893006003D534DA75340022C24020295D126604
:1028A300ED126701102A191559E55930E7158558B6
:1028B30059E558B4FF03755900D22A1266F1800E08
:1028C300855859E558B4FF0375590012671512A8C6
:1028D30087E5346003D534C12220106220115F7F65
:1028E300180548E54864187008F54830270375480B
:0B28F3000A121D3B303C2DDFE8802660
:1028FE0020105A2011577F181548E54830E7057506
:10290E004817800A64097006302703754817121D90
:10291E003B303C05DFE275480A121D6F1244C4E5D8
:10292E0032244C50051266BF800312668475340043
:10293E0002A8871229757F0EE5486B70048A4880BD
:10294E00020548121D3B303CD0DFED80CC122975BC
:10295E007F0EE5486A70048B4880021548121D3BB5
:10296E00303CB6DFED80B27A007B09E537B4030167
:10297E00227A0A7B17B40501227418FAFBF548D2A5
:10298E00362275A704758307E559C4F582E0E0F594
:10299E0073E0F574E0F575E0F576E0F577E0F5783F
:1029AE0075A7000244C4E5342437501A60391490D8
:1029BE00849B6013149084A2600D149084A9600708
:1029CE00149084B06001227F357E00124CC47F3398
:1029DE00122A080F122A087F3C122A080F122A0800
:1029EE000F122A0802A887908494204205204105E0
:1029FE0080D52041D290848C80CD7E2312A97CDE9E
:052A0E00FB12A97C226F
:1065590002660312AA5AE53724FD40F4E537B4026E
:106569000C304109E532248C50FA026C0E12A583D5
:10657900129B4B129BE7129D8012A07C7E197F36DD
:10658900129C7F12A38E129C95E537600514603525
:106599008054C23A12669A122F9F122D3230281D4A
:1065A900123027123196E5486418600CE54824F644
:1065B9005006201E0312327A12A91D801E1231962E
:1065C90012302780E1D23A1266ACC23C122A191263
:1065D900300A1297751296EE12A93512A6151243B2
:1065E90013124595800C1266A312965212A2251217
:1065F900A90D126BB0129C67800724FD401C12661E
:106609008475A70012A41A3022051229B4C22230B7
:106619002305122F78C22302A88712103712A43C2F
:106629007F1212979630124A75100075A704758368
:106639000612457DE51075F009A42415FFF5177EAE
:1066490000E512602F75F06484E5F00F129F0F1FAB
:106659007E0EE511129BA97516231246640510C317
:10666900E55A95104006E51024F550BF3012031283
:10667900672F808D745D129FBF80D5121037302926
:1066890008E548B418031210CA126740202A598035
:106699007B30120F30500C02696A301206200B034E
:1066A900026E6712A17120120122305106129AC29C
:1066B9000298B0029B1EE4FEFFE54824F6400D90C7
:0266C90084C18A
:1066CB00124CF57E16E548029F7AB40E069084C7ED
:1066DB00024CF59084CF124CF57E12E54824F7025C
:1066EB009F157D20800C7D3F302A077D633029026A
:1066FB007D3C7F0080247D2080127D3E800E7D3C82
:10670B00E54975F007A42406800A7D3FE55975F02D
:10671B0007A42409FF64027001FF7E1CED029F8D0C
:10672B007D2080027D3FE55B75F009A42416FF7E7A
:10673B0009ED029F8D9084D57E207F00124CF512BF
:10674B0066BF7E007F069067E9129FEDE5580460F7
:10675B005A75100075A70475830712457DE51075F2
:10676B00F007A42409FFF5177E00E512129F8D7820
:10677B0005EE2404FEE0129F8DD8F67920E030E779
:10678B0002792FE97E18129F8DE51230E70A90846B
:10679B00B87E20124CF5800A7E20E5111267B712E5
:1067AB0046C80510C3E558951050A92264B460245F
:1067BB0064B475F03284C0F0129F7ACE2404CED02C
:1067CB00E075F00584C0F0129F7ACE2404CED0E0A1
:1067DB0023029F7A9067E5024CF52D2D2D00014089
:1067EB00FFFFFFE0FFFFFFFFC25020093230122FE7
:1067FB0020282CE558F46027D25085591012682EAA
:0F680B0012687375A7049006DCE512F0E511F032
:10681A00E517F0E510F075A7049006E0ECF0EBF050
:10682A0075A7002275A70475830712457D7813E0C2
:10683A00F608B819FA9006D07811E6F008B819FAED
:10684A00E51CF516F0E51BF515F0758306E5102332
:10685A00541E24B0F582E0F513E0F5149006DAE54B
:10686A0014F0E513F075A70022120633E5BD75F0A2
:10687A0005A4D2F785F012F511E4F519FEF51CF519
:10688A001D128CA2C23DC2567F3C129828303D058B
:10689A00751900805ADFF3E5596558700A301007F8
:1068AA00EE24D35002D2568C1B8D1AE519FD24E230
:1068BA0050DEAE1CAF1D7C00123D6DEFF51924F6BB
:1068CA0050CEAC1BAD1A12976420D1238E048F05CB
:1068DA00E51975F0A7A4AEF0FF123D6D8F118E1267
:1068EA00C3EF94E8EE940340067512037511E7901E
:1068FA0006E2E519F012693FAC16AB157AC8123CEC
:10690A006FE512C2E7F9A811123E13ED7005EC24E7
:10691A009E50057C807B0822C3E57A305602E55CEE
:10692A009513FFE55E305602E55D9514FEC3EF9BB5
:01693A00FB61
:10693B00EE9CFC22AE16AF157C00E519FD24F6503B
:10694B001A123D6D7C007D06123C4D7C007D0512BC
:10695B003D6D8F10EEF51724E950037517FF2212CA
:10696B00978F12698212699C129D331269C2126948
:10697B00CD1269FF026A3A75A7049006D07811E030
:10698B00F608B819FA7F187E007812751907024DB0
:10699B004D75A7049006D8E0F516E0F515E0F51453
:1069AB00E0F513E0F512E0F511E0F517E0F510E076
:1069BB00FCE0FB75A700227F187E26AC14AB1302FC
:1069CB009DC17F2B7E009084DF124CF5E517F460A0
:1069DB0022AE17AF107C007D3C123D7AA805EF7FED
:1069EB002A7E0C129EC87E16743B129FBB7E18E843
:1069FB00129EC222E51233923BC313FEAF117C00F1
:106A0B007D0A123D7AA805EF7F207E30129EC87E4C
:106A1B003A742C129FBF7E3CE8129FA57E29203B27
:106A2B00060F7445029F8D7467029FBF026AEB12BB
:106A3B006B5EC23DE54824F640F2E559046558709B
:106A4B00EBA217923D8E1E8F188515179006D0E07E
:0F6A5B00F5118558101510123176C3E5119510FD
:106A6A005002F404F924A65005C374B399F9E975E0
:106A7A00F00584F924EE50027911906B9EE993F5A2
:106A8A00F012063DE5BD23A4A9F0E51B2517FDE597
:106A9A001C3516FEC3ED99F515EE9400F51675A78B
:106AAA0000758306E55823541E24B0F582E0A3F549
:106ABA0013E0F514126B5E20170C203D1AC3EF95F4
:106ACA0018EE951E401175A7009006E0E516F0A392
:106ADA00E515F0D23D800AA23D9217AE1EAF18C24C
:106AEA003D7C007D0A123D7AA805EF7F2A7E30128E
:106AFA009EC87E3A742C129FBF7E3CE8129FA52046
:106B0A003D10E54824F64006E55965586004746C62
:106B1A008007746E205602746D7E28129FBF30174C
:106B2A0007742D7E3A129FBF203D0122855810120C
:106B3A00682E12698212699C8C168B151269C21210
:106B4A006902126820129D339006E2E0F519126973
:106B5A003F0269CDC3E57A305602E55C9513FFE53D
:106B6A005E305602E55D9514FE92175003123EE41C
:106B7A00AC16AB157AC8123C6FA906A807123E13C9
:0A6B8A007E037FE7ED700CEB24188A
:106B9400EC34FC4004AE04AF032200172E43576CC0
:106BA4008092A4B6C5D3DFE6EDF3F8FD30504C7502
:106BB400A7009006E0E0A3FCE0FBECA2E7921740FC
:106BC4002024FE50047F3B8022AE04AF037C007D72
:106BD40014123D7A74542F2017029F9FFF74628011
:106BE4000C123EF4EC24FE50E07F6D743D7E0012E6
:106BF4009F8D7E017D197C03126C00227F3D12A9BA
:106C04004CEF2DFFDCF82212AA5A12A583129B4BDB
:106C1400129BE7126D7A12962112A0FD12A91D1281
:106C24006DD21245957F207E2B129C7F12A38E126B
:106C3400A41A126CB302A887E579FD24A050027D42
:106C44005FED24CD401E744520750C2DFFF5121206
:106C54006C881FBF44F922C39DFFF512126C880F84
:106C6400BF46F92220750EED2413FFF512126C882D
:106C74000FBF78F922C374779DFFF512126C881F39
:106C8400BF12F922EF24BA40082433FCC374329CA7
:106C94001404FC24D750047C238009EC2375F005EC
:106CA400842413FC7E0512A94C0EECB506F82212BE
:106CB4006C3C7F457E047D0E12A94C0EDDFA7F43A9
:106CC4007E007464129F8D7F4F7D12126D637F3B33
:106CD4007D12126D637F597D16126D637F317D16AF
:106CE400126D637F637D1A126D637F277D1A126DA7
:106CF400637F6D7D1E126D637F1D7D1E126D637E2D
:106D0400057F1912A94C0FBF72F97804E57924CDD7
:106D140050027809E8305C0123F87F1B126D527F22
:106D24006B126D5218305C01187F25126D527F6111
:106D3400126D5218305C01187F2F126D527F57125A
:106D44006D5218305C01187F39126D527F4D7E00F0
:106D5400E875F00A847004E8029F7AE8029F15EF50
:106D64006512600C7E04EE20E00712A94C0EDDF6DD
:106D74002212A97C80F7907F2F7F287E2C124CF55D
:106D84007E3B129DD8AC5EAB7A7F307E19C23D1239
:106D94009E179084E37F5D7E2D124CF578B9C3E590
:106DA4007A9618FBE55E96FC7F507E19D23D029ED2
:106DB40017E51164B4700122E51112A8277831791E
:106DC4000F7D0B12A8D01F1E906E62029FEDE5711D
:106DD4006012E57012A8277831790F7D0412A8CCCF
:106DE4000DBD0AF97F01126E3A7F1D126E3A7E23A1
:0F6DF400126E447E3F126E447E247F17126E4E45
:106E03007E397F02126E4E7E247F07126E587E39C2
:106E13007F1C126E587E317F0212A94C7F1C12A96F
:106E23004C7F0F7E2412A94C7E3E12A94C7F0C7E10
:106E33002E90A69B029FED7E2A12A94C0EBE39F915
:106E4300227F0812A94C0FBF17F9227D0612A94C05
:106E53000E0FDDF9227D0612A94C0E1FDDF9220368
:106E630003E0A0E012978F7F187E009084E9124C14
:106E7300F57F217E017441129F8D7F2A7E01745319
:106E8300129F8D9005BEE0F51AA3E0F519A3E0F576
:106E93001EA3E0F51D851A1C85191B751720126F9B
:106EA3001AE519251DF51BF51DE51A351EF51CF50B
:106EB3001E751729126F1A9005BA126F0AAC1AAB16
:106EC30019751720126ED79005BC126F0AAC1EAB52
:106ED3001D751729EC7007EB249B400280287A4824
:106EE300305D027A27123C6F123E13ED4C7017AFE0
:106EF300177E07EB129E740F7E1A9084F9305D03A0
:106F03009084FC124CF522E0FEA3E0FD128DFCC33D
:106F1300EB9DF8EC9EF9227516271247161246913F
:106F2300AF170F7E379084FF305D03908502024CCC
:0F6F3300F5128DFC75A7049005B478737F06E600
:106F4200F008DFFBECF0EBF0E0E0E0FCE0FDE0FE5F
:106F5200E0FFEF2DFFEE3C9005C0F0EFF0801275E0
:106F6200A7049005BAE0FBE0CBF0EBF0E0E0E4F040
:106F7200F075A7002275A7049005B478647F06E037
:106F8200F608DFFB75A70012473D9005BEE51CF031
:056F9200A3E51BF02245
:102A1300D23C799E7700128CA2E4F510F511F512E1
:102A2300F513F514F515F516F517C23D122BDC2039
:102A33003D1F122BDC203D19E51F30E51130E40E5C
:102A4300122A86303C08799EE724F5500122D510DE
:102A5300DBAE14AF157C00AD12123D478F55AE1699
:102A6300AF177C00AD13123D6D123F6E7E00E5552E
:102A730030E7011E2DFFE43E30E7027F00740A2F8A
:102A8300F55622C235E51CAF1DBFFF050FD235F445
:102A930004FABF003F752C00E518AF19BFFF050FFF
:102AA300D262F404BF002D20E72A205B0123FF2418
:102AB300AA4021E51AAE1BBEFF050ED261F404BE87
:102AC30000128547F0A4E5F020E709205B0123FE0F
:102AD30024AA5001227C567B1F305166302163C0EB
:102AE30006C0078AF0E545A4AEF0FFE556205B017A
:102AF3001375F009A4ACF0FD123D6D74FFBE000127
:102B0300EFFA24C050027A3FD007D006E55212A84C
:102B130027303504B2D5B2D1EA8CF0A430E70205F0
:102B2300F0745625F020D10495F095F0FCEA8BF073
:0A2B3300A430E70205F0741F25F03E
:102B3D0030D50495F095F0FBEC2F2062029F9FFF9E
:102B4D0024884017EF24CB5012EB2E3061029E9E4D
:102B5D00FE24C04006303C04799E072212A94CE5A4
:102B6D001E24FB50F60E12A94CE51E24F650EC1E49
:102B7D001F12A94CE51E24F150E11E0F12A94CE5C0
:102B8D001E24EC50D60F12A94CE51E24E750CC1F85
:102B9D001F0E0E12A94CE51E24E250BF1E0F0F1280
:102BAD00A94CE51E24DD50B30E12A94CE51E24D808
:102BBD0050A91E1E1F1F02A94C128BCD128ACAE4EA
:102BCD00F5F7C2B2C2B2E5F7D2B2C22064C022207C
:102BDD003D07122BC67003D23D22056D056D128A7D
:102BED00CA7D008DF7C2B2C2B285F71F8DF7C2B292
:102BFD00C3E5F79573F5188DF7C2B2C2B2E5F79537
:102C0D0074F5198DF7C2B2C2B2E5F78DF7C2B2C332
:102C1D00E5F79576F51A8DF7C2B2C2B2E5F795775D
:102C2D00F51B8DF7C2B2C2B2E5F78DF7C2B2C2B2D3
:102C3D00E5F7F51E8DF7C2B2C3E5F7957AF51C8D54
:092C4D00F7C2B2C2B2E5F78DF73F
:102C5600C2B2C2B2E5F7D2B2C220543F30E5024456
:102C6600C0955EF51D156D156DE5102478400122A1
:102C76007E00AF55EF30E7011E0512E51FA2E59273
:102C8600D5400EE515951EF515E5149400F514804E
:102C96000BE515251EF515E43514F5147800E51E2B
:102CA600600620D50318F404C39FF5F0E89E30E7CC
:102CB60001220513E5F0A42517F517E5F03516F5FD
:102CC6001622303D03D23D22122BC660F8122BC6C7
:102CD60060F3E546600A122BC660EA122BC660E571
:102CE600056D056D056D128ACA7D008DF7C2B2C3EA
:102CF600E5F79573F5188DF7C2B2C2B2E5F795748C
:102D0600F5198DF7C2B2C2B2E5F78DF7C2B2C3E5C7
:102D1600F79576F51A8DF7C2B2C2B2E5F79577F553
:102D26001BD2B2C220156D156D156D2230122220F0
:102D36000F1FE5467A0260077A06146002801212B7
:102D46008CA2C23D7878122CC8203D05122D58D889
:102D5600F522752C00E518AF19BFFF050FD262F4F6
:102D660004BF002A8AF084FF24DF4022E51BA2E785
:042D760013FEE51A49
:102D7A0013BEFF050ED261F404BE000E8547F0A40F
:102D8A00EA03C5F084FE24E050012274562F206223
:102D9A00029F9FFF741F2E3061029E9EFE02A94C65
:102DAA0074542F2062029F9FFF741D2E3061029E71
:102DBA009EFE2279B4203245201D42EFB5060092CC
:102DCA0060AC06AB074004AC07AB06902E08EC23B8
:102DDA0004938BF0A4A9F0EC23938BF0A429F99027
:102DEA002E6893C9902F68E52C9313E95001F4904B
:102DFA002F70F9E52C932975F0B484A9F022FFFF0E
:102E0A00FFFF7FFF55553FFF33332AAA24921FFF46
:102E1A001C7119991745155513B1124911110FFF54
:102E2A000F0F0E380D790CCC0C300BA20B210AAA0D
:102E3A000A3D09D8097B092408D30888084207FFF4
:102E4A0007C107870750071C06EB06BC06900666F3
:102E5A00063E061805F405D105B005900572000076
:102E6A000000000101010101010101010202020247
:102E7A00020202020203030303030303030304041B
:102E8A0004040404040404050505050505050505EF
:102E9A0006060606060606060606070707070707C2
:102EAA000707070808080808080808080809090998
:102EBA00090909090909090A0A0A0A0A0A0A0A0A6F
:102ECA000A0B0B0B0B0B0B0B0B0B0B0C0C0C0C0C44
:102EDA000C0C0C0C0C0C0D0D0D0D0D0D0D0D0D0D1E
:102EEA000D0E0E0E0E0E0E0E0E0E0E0E0F0F0F0FF5
:102EFA000F0F0F0F0F0F0F0F1010101010101010D0
:102F0A0010101010101111111111111111111111AC
:102F1A001111121212121212121212121212121388
:102F2A001313131313131313131313131313141465
:102F3A001414141414141414141414141415151544
:102F4A001515151515151515151515151516161624
:102F5A00161616161616161616161616161600FF34
:102F6A00FF00FF0000FF002EB5875B2D5A88E5346D
:102F7A0024374001227F357E2B7D0F600C7D1E1485
:102F8A0060077D3C1460027D78ED305D02C3131248
:102F9A009E7402A887E546604A14603C14602E14A9
:102FAA00602014601290852D205D419030207F367C
:102FBA007E34129FED803C90852D305D03908529EB
:102FCA00802A908529305D03908525801F9085256C
:102FDA00305D039085218014908521305D039085B2
:102FEA001D8009908519305D039085157F367E33E3
:062FFA00124CF51F7E3CA5
:103000007422305D027466029FBF305D08908505B2
:10301000305BE3800690850D205BDB90850980D6D0
:103020000508B28D8DB5BAE558B4FF012278007558
:10303000A7047583071231F188188A1E8E168F1720
:1030400030D15AC23EE54824F6404FD23EE55860A2
:1030500049E865597044E54624FE403B75F0360466
:10306000700375F01212063DE5BDB80002E5BC60C4
:1030700026A4ACF0FB123E83123E83EBFDF5111249
:1030800030AA1230B6E51865587009E54670057D1E
:10309000061230B61230F412312C1230CCA81808B7
:1030A000C3E55898508975A70022122DAAEE240274
:1030B000F8EF2402F9227A00EA12A82712A8D00A0F
:1030C0000AED24F440020A0ABAB4ED22AE16AF1794
:1030D000122DAA1E303E021E1EE51E129F8DEE24EA
:1030E00004FEE512129F8D303E09EE2404FEE51326
:1030F000129F8D22E51865586031851810C012C0E6
:1031000013123176D013D012E51012A827AE16AFE5
:10311000171230AAE511FD24F840027D080DEDC319
:1031200013FA12A8D01DC3ED9A50F722200C40E5E7
:0331300018703CD8
:10313300F510C012123176D012E510247940022422
:10314300B412A827AE16AF171230AAE54624FA40E8
:103153001BE54690317093FD12A8D0B2D5B2D112BF
:10316300A8D0B2D5B2D11DED24FD40EC225A592D81
:10317300160B0612961575A7047583071245501290
:10318300960F0510124550C02C124569D02C89109A
:1031930002961B20120122780075A704758306127C
:1031A30031F130D139122DAAE54624FE500A0E0F13
:1031B3009031EC129FED8026EA7007745D129F89AF
:1031C300801C75F06484ADF0700FED75F00A8470A7
:1031D30008E5F00E129F7A80051EED129F0F08C3BB
:1031E300E55A9850B475A70022030340A040D2D1FA
:1031F300E8C4F582E0FA797312324A30D146AF0659
:10320300752C00EDBFFF07F40460390FD262BF00D5
:1032130033123370402E797612324A30D126E5824A
:103223002403F582E0F512E0F513EEA2E713FEEDB9
:1032330013BEFF07F404600C0ED261BE0006123306
:103243008D400122C2D122C3E09709FDE09709FE18
:0B325300E097600904700AEE30E70607
:10325E008007EE30E703C2D122E546600E14600B04
:10326E00F9EDCEA2E713CE13D9F8FD227C007B44F4
:10327E00E54660207C007BCC1460197C017B9814A1
:10328E0060127C037B3014600B7C067B6014600440
:10329E007C0C7BC08C148B157AE9123C6FA84712FC
:1032AE003E118C168B1775C70075C6047510DF7529
:1032BE00B901E5BC20E76FF51385BD1205C605C63D
:1032CE0075B901752C00C3E5BE9573FBE5BF95740A
:1032DE00FC05C675B901E5BC9575FD5005D26212A7
:1032EE003EFCC3E5159BE5149CE49D40338C198B85
:1032FE0018C3E5BD9576FBE5BE9577FCE5BF9578E1
:10330E00FD5005D261123EFCC3E5179BE5169CE409
:10331E009D400D8C1B8B1A123345E5322428401329
:10332E0005C6E5C68006E5C62404F5C6700205C7C7
:10333E00D51001220232BDAE19AD18123267ED1250
:10334E003370AE1BAD1A123267EE13ED1312338DBE
:10335E00122DAA1EE513129F8DEE2404FEE5120215
:0C336E009F8D75F0067FFDA946B9000593
:10337A0075F0027FFF84C5F02F500205F0C5F0FFFB
:10338A0024DE228547F0A430E70205F0E5F0A946DD
:10339A00B9000280050475F00384FE24E022E537B3
:1033AA00B40203204119E5377002D239640270026F
:1033BA00C239E53724FD799EE76005640B600C226B
:1033CA00D27E20081E401C107F1022D27F200813B4
:1033DA004011107E0122753701227537002039030A
:1033EA007537022220532712343D759E85759D2D0F
:1033FA00C2AC759852C26DC26EC26F221233F17599
:10340A00F9FF2212343D759E84759D2D80E275F96F
:10341A00FF75FBFF800312343D759E83759D0980FD
:10342A00CF12343275FBFF2212343D759E82759D90
:10343A000980BDE4F5F9F5FB22D2A412A9B7C2A40A
:10344A0012A4E712A88712A9ACD220C214C215127C
:10345A00340674C012A74B74A312A75D748F12A707
:10346A005DE53812A75D74CA12A75DC2202275A64F
:10347A000A123453D269D2ACE5A624FA500C306D44
:10348A00F712A7E4B4E0F11234BEC2ACC26975A661
:10349A00FF22D21EC274C273E4FDF571F5701234B4
:1034AA0006D2AC12A7E4C5F07005DDF7C2AC22C59E
:0934BA00F0B4E0EFF538E4F5325E
:1034C300C274C27375A7049004B412A7DAF0A2E21F
:1034D3009274A2E1927312A7DAC2D112368C2069D8
:1034E3000330740B8D758E748F73E514C4F57D12E0
:1034F300370C12368C20690330740C8D788E778FDD
:1035030076E514257DF57D12370CD2D112368CEE7B
:10351300F0F55DEFF0F55C12A7DA7D0A1236F98F4C
:1035230071EE60037571FF7C007D05123D7A8F514A
:103533007D141236F98F7012A7DAF05407C52E5492
:10354300F8252EF52E75A70012A7DAE5386009D203
:103553001EC27412779E8005C21E12779A12A7DAD2
:10356300B4E1FAF53875A7049004C412A7DAF0128F
:10357300A7DAF0F53A12A7DAF0F53B12A7DAF0F57D
:103583003C12A7DAF0F53D12A7DAF0F53E12A7DAFE
:10359300F0F53F12A7DAE538600674C59004C8F069
:1035A30012A7DAB4E2FA12A7DA9004CBF07E0C1277
:1035B300A7DAFF12A7DA12A7DA12A7DA12A7DA201C
:1035C300E1027F00EFF012A7DADEE412A7DAB4E338
:1035D300FA12A7DAFF12A7DACF60027F7F9004E422
:1035E300EFF0E4F012A80F9004D81236F912A7DA1C
:1035F300B4EAFAC2ACE561F0E560F0E55EF0E57AC5
:06360300F0E579F0E52E70
:10360900F0E55FF0E57BF0E57EF0207412E49004CC
:10361900B4F09004BDF0F0F0F0F0F0F571F57075CC
:10362900A70078ABA63A08A63B08A63C12063DE5DA
:10363900BF253D240C75F0188478AEA6F0186005F6
:10364900640260182216E670121816E67004760CE9
:10365900181678ACE690367F9308F6220618E60825
:1036690090367F930466700D76011806E6640D7036
:10367900047601180622001F1C1F1E1F1E1F1F1E75
:103689001F1E1F12A7DAFC12A7DAFD12A7DAFE1213
:10369900A7DAFFECA2E692E7921713FCED92E71383
:1036A900FDEE92E713FEEF92E7301701F4F513EC04
:1036B900A2E713FCED92E713FDEE92E7301701F450
:1036C900F512ECA2E713301701F4F510ED92E7308B
:1036D9001701F4F511123EA420D10E8C1C8D1D8EFC
:1036E9001E8F1F127BA6123EA4301703127B802265
:1036F90012A7DAC313FEF012A7DA92E7FFF07C00F3
:05370900023D7AAC1C3A
:10370E00AD1DAE1EAF1F301703127B80ECF0EDF037
:10371E00EEF0EFF02212372C02026E128A51D220F6
:10372E0012347B7F367E05908531124CC412A887E9
:10373E00D214C255121ED8789F7680087600128A4F
:10374E007812243B7570FE853A71853B72853C7309
:10375E00853D74853E75853F76128B6712243B75C9
:10376E0070C0757B03757A54E4F57FF57E128B6716
:10377E00751421751348755F01757B007575047599
:10378E00745275780175776CE4F57DF57E757F0161
:10379E0090D63485836E85826DC23D123808851CA5
:1037AE001D75A6FF3055097554B5121FC1C22022D2
:1037BE00123808E572A2E59275A2E79277D274D21A
:1037CE0073E51275F008A4AEF0FF207503123EE407
:1037DE001295801295C412388BE51C251D13F571B8
:1037EE00851C1D128A89128B1F757F027F367E35CE
:1037FE00E541129E5712A88780A7856E83856D823C
:10380E00C255787312386C787612386CE493F57072
:10381E00B4B402D255A3E493F51CA3E493F512A31A
:10382E00203D0FA97BE493F57BC399502A20E70234
:10383E00055FA385836E85826D103D16D23DE582B0
:0D384E002405F582E43583F583E493F52627
:10385B0054F0F57222E526C480F630E7D8155F8068
:10386B00D48601E493F6A308C399500A20E7060611
:10387B00B6000208062230E70616B6FF021816221B
:10388B0030750DE5132579F513E43514F514800D1A
:10389B00C3E5139579F513E5149400F514AE14AF45
:1038AB00137C007D0A123D7A8E5E8F7A2275C703D8
:1038BB0075C6FC128A6A75BC261239E475C6FA7590
:1038CB00BC1475BD1475BE0075BF0C1239E475C6FA
:1038DB00F875BC0A75BD0F75BE0075BF050239E4DE
:1038EB00120651E5BC0460637F5D7E0890845B1219
:1038FB004CC47E20E5BC129FBF7E26E5BD129FBF48
:10390B007E2CE5BE129FBF7E32E5BF129FBF02A881
:10391B0087D23D7F3F7E297513501239437513486B
:10392B0012394375135012394375134B1239433007
:10393B003D0312395602026EC224785F1259DBE83E
:10394B0065136002C23DEE2406FE22C210C2117541
:10395B00B9061238B81239EF12A9AC75C70375C680
:10396B00FF7430128A6F75BC341239E41238F312BB
:10397B00104B751303800C75A6FF7E20A8BC125943
:10398B00D788BC7F747E36E51314129F7AC23C7FB6
:0E399B005D7E26A8BD1259D788BD7E2CA8BE21
:1039A9001259D788BE7E32A8BF1259D788BF303C7A
:1039B90003751303D513C275C70375C6FF1239E41E
:1039C900123453128A51123B7412372C75C6F97589
:1039D900BC0E75BDFC75BE0075BF10D22075B9054A
:1039E90075B902C22022123453D2AC75A6FF12AAAD
:1039F9005A100067306DFA12A7E4B4E2F412A7DA9C
:103A0900F51375120C75110612A7DAD511FA60159E
:103A1900F42460FFE51275F005A4FE12A94C0FC34A
:103A2900EF944740F6D512DD7F287E0E908542122D
:103A39004CC4E513129E5D7F321297967F4612970A
:103A4900967F147E1212A2297F027E0B90853A126C
:103A59004CC412104612A887300290C202C2AC228E
:103A6900D214E4F56CF56BF56A12AA5AE4FEFFE587
:103A79006C129E747E14E56B129E747E28E56A545E
:103A8900C0F56A129E74751E00751F04128C4912C6
:103A99008B827F0A7870E608AE1E129F2BEF2407EF
:103AA900FFB880F2E51E2410F51ED51FDF12A88786
:103AB90075A6FF10000610020280F5221002FCC252
:103AC9003D7904128C49128B82E57064FF6008E528
:103AD90070244C5002D23DE57F24FE4002D23DD9EC
:103AE900E2303DD87904128BB0D9FB023A72D21474
:0C3AF90012AA5A75C70375C6F0E4FEFF60
:103B0500E5C7129E747E14E5C6129E74751F107F5C
:103B15000A75B9017E00E5BC129F2B7E10E5BD122A
:103B25009F2B7E20E5BE129F2B7E30E5BF129F2B7B
:103B350005C6EF2407FFD51FD8E5C624F0F5C61244
:103B4500A88775A6FF10001710010510022080F246
:103B5500E5C62410F5C670A505C753C703809EC3E7
:103B6500E5C69410F5C6E5C79400F5C780EC22E4D8
:103B7500F5C7F5C675B90505C6E5C664E06008E58F
:103B8500C670F105C780EDE5C7640370E7123B9881
:103B9500025142E4F5C7F5C67426123BA9123BA9AA
:103BA500E4123BA9128A6F1239E405C6227F5D7EB5
:103BB5000DE56C129F2B7E1EE56B129F2B7E2FE56C
:103BC5006A029F2B7F3C7E00E54B129F2B7E10E502
:103BD5004C129F2B7E20E54D129F2B7E30E54E0229
:023BE5009F2B14
:10D6340069FC362E06FD69FC372F071169FD383069
:10D6440007FD69FD3931061169FE383107FD68FEB1
:10D654003732091168FF373008FD68FF372D07118D
:10D664006800362909FE680036290C116801372B39
:10D674000CFF6801372F0A116802383009FF68026D
:10D68400372E08116803372C0AFE6803372E081159
:10D694006704373208FE67043633091167053535E8
:10D6A40005FF6705353303116706362F02FF67064A
:10D6B400362B05116707362B07FF6707352F051132
:10D6C4006708353104FF6708332E051167093128CF
:10D6D4000700670931250A11670A35240B01670A17
:10D6E4003A240A11660A3C210801660B3D1E0B11FF
:10D6F400660B3D1E0C00660B3D200A11660C3B2197
:10D704000CFF660C39220E11660C37231100660DCE
:10D7140036240D11660D34260F01660E32261111C2
:10D72400660E32251401660F35251311660F37274F
:10D7340016016610392918116610392B1502651166
:10D74400392D11116511372E0C026512332F081172
:10D754006512312F07026513302C0A1165132D2928
:10D764000E0265132A271011651429270E02651469
:10D774002C290C1165153129080365153726071165
:10D784006515321F09036516411B09116516411CF5
:10D7940008036416461F081164164D210504641617
:10D7A4005922031164166425040563156A240711BC
:10D7B40063156D23090663156C230D1163156C2520
:10D7C400130762146E2B151162146E2F1406621364
:10D7D4006E30161162136E30150761136F3112111A
:10D7E40061126F350F0761126F380D116011723AB3
:10D7F4000A086011763F0611601079420209600F31
:10D804007A3A0533600F7832040A5F0F742C0133BF
:10D814005F0E722B030A5F0E732E08115F0E7430B5
:10D82400050C5F0D722C02135E0D6C2B010C5E0D4A
:10D83400622C05315E0D5F2B030D5D0D5E290833EF
:10D844005D0D5F23030B5D0D5F1B01335D0D5A16E8
:10D85400020A5D0D521B00115C0D4D26000C5C0E7E
:10D86400462802335C0E3926040C5C0F2C2B08333B
:10D874005C0F23320C0F5D0F172E0A335D0F0C2E35
:10D8840009105D0F043507335E0FB23C080F5F0FBC
:10D89400AB4209335F0EA43E070F5F0EA2430B3366
:10D8A400600EA746120B600D9F490C73610C9C49D6
:10D8B4000F0C610B97460973610B8B440A0C610AC8
:10D8C4008B420B336109843A080C6108823A0433B1
:10D8D40061087934030C60086F2F063360086228EE
:10D8E400050C6008572505336008511F040D5F08B7
:10D8F4004E1B05335F08491B090D5F094120103792
:10D904005F0938270D0D5F0A302F06335F0B2B326A
:10D91400070F5F0B282F0A335F0B262E0E0E600CA9
:10D9240023361137600D1F3F160F600D1841127713
:10D93400610D0F320A13610D042B0633610D022EA3
:10D94400040E620D043A0231620E0343050D630DA9
:10D95400B1470113630DA94A000B640CA14D0511D5
:10D96400640C9B44070E650B99490911650A944799
:10D97400090D65098E49021365088848060D650876
:10D9840081400E336407793B130F6407722F1877B5
:10D9940064076D231A106407692911776407651CED
:0DD9A400080F63075D180B33630751190D61
:10D9B1000D630746220E336308402B110F630838AD
:10D9C100291837630932271B0D6309312B1477623C
:10D9D1000A372C0F0A620A3C280973620A441E0B9B
:10D9E1000C620A48150E33620B46190C0A620B478A
:10D9F100260D33610B4C280C0B610B54251037613C
:10DA01000B5E24170C600B63291A77600A663614C3
:10DA11000A600A68390B735F0A6C2C100A5F09727D
:10DA21002015775F097422120A5F0873300F775F40
:10DA3100087639140A5F077D3816775F0785370F37
:10DA4100095F068D3B0D735F058B4410075F048BE7
:10DA5100490C735F048E3F0C075F03863604335F06
:10DA61000394280708600299300E1160029E400558
:10DA7100076102A34A0C336101AA4810086201B18F
:10DA810042127762020131150A6202062B13776393
:10DA9100020830110C63020B361277630310331145
:10DAA1000C6403182B147764032223110A640426DF
:10DAB10023107764042226110A64051C2715776454
:10DAC100051D251508640521271277640628270FEF
:10DAD1000764062F1D11776406350F140764063E8F
:10DAE1000A19776406401216086407431B1177630D
:10DAF100074A22120663075228127763075A27132F
:10DB01000662075E231477620661201107620664CC
:10DB11001E0E7362066A1E0E0762067421103762BA
:10DB2100057828130661057A2F157761047A332069
:10DB31000661047A301B7761037A281B0761037F32
:10DB410023187761028429160661028832177761EA
:10DB5100018D371305610193340C7362009A2E090C
:10DB61000562009D2E043362009D370C0663FFA001
:10DB710040103763FFA844140564FFAF4612776471
:10DB8100FF014511056500043F12776500053E1050
:10DB9100076600073F117766000B430D0767011009
:10DBA1003D117367011539120767021A321277673F
:10DBB100021A2C12076702192C107768031B2E0F0B
:10DBC1000668031F2C117768042729100468042EA6
:10DBD1002A0F776705322F130467053330127767F1
:10DBE10006362D140567063B291677670643231B66
:10DBF100046706471E16776607491E150366074C1C
:10DC01001B157766074C22170466075222147765A5
:10DC1100075B26150265066229157765066D2917CA
:10DC21000165067529137765057D281A0265058248
:10DC310028187765047F1F160265048F2A117765FE
:10DC410003953211006602993D157766029C401CCE
:10DC5100FF6602A13E1F776701A43F1CFF6701A772
:10DC61004314776801AB4710FF6901B1490F776928
:10DC710001024911026A0207490D736A020B480C3D
:10DC8100056B030F480B336B03144A0D026B041928
:10DC91004914376B051F491CFE6C06224824776C1A
:10DCA10006233F21FC6C07203023776C07212721B5
:10DCB100FC6C07262420776C08292812FC6C0828A4
:10DCC1002C0F776C0927230CFF6C09251802316C86
:10DCD10009350F05FC6C094C1401116C09561D0125
:10DCE100FC6B095F2003136B086B2108FB6B087445
:10DCF1002509336B08772507FC6B0778210D336BFA
:10DD0100077A1E0AFB6B077F220C336B06832E0AF0
:10DD1100FA6B05853C09336B0489410EF96B048C60
:0DDD21003E10376B038D3C0FFA6B038D40F5
:10DD2E0013776B02904112FA6C01934110776C01DC
:10DD3E00984410F86C009B471A776D009F461EF8AA
:10DD4E006DFFA24519776EFFA14019F86EFFA64030
:10DD5E0014776FFEAA4417FA6FFEAF4A127770FE61
:10DD6E00B34D18FA70FF024B1B7771FF054718FD74
:10DD7E0071FF0942177772000E4012FD7200163DB8
:10DD8E000C7372011B3510FA7201232E1577720275
:10DD9E0029321AF872032C371D7772032F3014F8BC
:10DDAE00720336210F77710346190DF87103502057
:10DDBE000B33710353290EF87003572B143770036E
:10DDCE00612712F870036F2911777002793017F7F7
:10DDDE007001803722777001843D1FF67000883FF6
:10DDEE00197770FF8D3F11F670FF933D0C7371FE26
:10DDFE00973D0EF571FE9B3E0C3372FD9F4310F660
:10DE0E0072FDA448127773FDAB4C13F573FDB14F41
:10DE1E00167774FD034F14F775FE074C127775FED7
:10DE2E000A4510F975FE0E400F7776FF124111F874
:10DE3E0076001745167776001C4614F676012142B9
:10DE4E0017777602263D17F3760229382177760367
:10DE5E002A3315F276032B3009737604302A07F035
:10DE6E00760439220A337604472110F075045125C1
:10DE7E0012777504552416F1750459210F77750420
:10DE8E005F2111F0740463231477740468240EF276
:10DE9E00740370230933740379270AEF74028030F8
:10DEAE000B33740185360DEF74018B391337740003
:10DEBE00903D1BF075FF94441E7775FF984823EF35
:10DECE0075FE9B46207776FE9F4221F076FEA13F9F
:10DEDE00177777FDA44313EF77FDA747157778FDE6
:10DEEE00AA4915EF78FDAD4C157779FDB04D19EEB9
:10DEFE007AFDB34D1C777AFD024E19F07BFD054F6E
:10DF0E001B777BFE094F24F37CFE0D531D777CFFA0
:10DF1E00114619F37CFF173F12777C001F3810EF64
:10DF2E007C00263613777C012B3115ED7C012F2BCF
:10DF3E0015777C02332513ED7C02392214777C028F
:10DF4E00402110EE7C0249210B737B02531F0FEB15
:10DF5E007B02601E15777B026A2214EA7B0174280D
:10DF6E0019777B017B2D1AEA7B00833122777B00A8
:10DF7E008A3320EB7BFF91371A777BFE953C1FEAA5
:10DF8E007CFE983C26777CFEA74621EC7CFD9939D9
:10DF9E0023777CFC9A3B1FEA7DFC9A3F1C777DFB26
:10DFAE009A401EE87DFB9B3F20777EFA9B3F1FE643
:10DFBE007EFA9C431A777EF99E4717E57FF8A04AB2
:10DFCE000E737FF8A34A0AEA80F8A548073380F853
:10DFDE00A94402EA81F8AE46041182F8B24C00E779
:10DFEE0082F80351021183F8085304EA83F90E4DA7
:10DFFE00061183F914430CEC84FA1A400E1184FBBB
:10E00E00203F0AE884FC2540061384FC2B4008E6DA
:10E01E0084FD3039073383FD36300EE483FE3C2B0E
:10E02E00193783FE402A1EE783FE3D25187783FEAF
